ARM Linker, 5.03 [Build 76] [MDK-ARM Standard]

==============================================================================

Section Cross References

    startup_stm32f40_41xxx.o(STACK) refers (Special) to heapauxi.o(.text) for __use_two_region_memory
    startup_stm32f40_41xxx.o(HEAP) refers (Special) to heapauxi.o(.text) for __use_two_region_memory
    startup_stm32f40_41xxx.o(RESET) refers (Special) to heapauxi.o(.text) for __use_two_region_memory
    startup_stm32f40_41xxx.o(RESET) refers to startup_stm32f40_41xxx.o(STACK) for __initial_sp
    startup_stm32f40_41xxx.o(RESET) refers to startup_stm32f40_41xxx.o(.text) for Reset_Handler
    startup_stm32f40_41xxx.o(RESET) refers to stm32f4xx_it.o(.text) for NMI_Handler
    startup_stm32f40_41xxx.o(RESET) refers to stm32f4_discovery_audio_codec.o(.text) for DMA1_Stream0_IRQHandler
    startup_stm32f40_41xxx.o(.text) refers (Special) to heapauxi.o(.text) for __use_two_region_memory
    startup_stm32f40_41xxx.o(.text) refers to system_stm32f4xx.o(.text) for SystemInit
    startup_stm32f40_41xxx.o(.text) refers to __main.o(!!!main) for __main
    startup_stm32f40_41xxx.o(.text) refers to startup_stm32f40_41xxx.o(HEAP) for Heap_Mem
    startup_stm32f40_41xxx.o(.text) refers to startup_stm32f40_41xxx.o(STACK) for Stack_Mem
    system_stm32f4xx.o(.text) refers to system_stm32f4xx.o(.data) for SystemCoreClock
    stm32f4xx_adc.o(.text) refers to stm32f4xx_rcc.o(.text) for RCC_APB2PeriphResetCmd
    stm32f4xx_can.o(.text) refers to stm32f4xx_rcc.o(.text) for RCC_APB1PeriphResetCmd
    stm32f4xx_cryp.o(.text) refers to stm32f4xx_rcc.o(.text) for RCC_AHB2PeriphResetCmd
    stm32f4xx_cryp_aes.o(.text) refers to stm32f4xx_cryp.o(.text) for CRYP_KeyStructInit
    stm32f4xx_cryp_des.o(.text) refers to stm32f4xx_cryp.o(.text) for CRYP_KeyStructInit
    stm32f4xx_cryp_tdes.o(.text) refers to stm32f4xx_cryp.o(.text) for CRYP_KeyStructInit
    stm32f4xx_dac.o(.text) refers to stm32f4xx_rcc.o(.text) for RCC_APB1PeriphResetCmd
    stm32f4xx_gpio.o(.text) refers to stm32f4xx_rcc.o(.text) for RCC_AHB1PeriphResetCmd
    stm32f4xx_hash.o(.text) refers to stm32f4xx_rcc.o(.text) for RCC_AHB2PeriphResetCmd
    stm32f4xx_hash_md5.o(.text) refers to stm32f4xx_hash.o(.text) for HASH_DeInit
    stm32f4xx_hash_sha1.o(.text) refers to stm32f4xx_hash.o(.text) for HASH_DeInit
    stm32f4xx_i2c.o(.text) refers to stm32f4xx_rcc.o(.text) for RCC_APB1PeriphResetCmd
    stm32f4xx_pwr.o(.text) refers to stm32f4xx_rcc.o(.text) for RCC_APB1PeriphResetCmd
    stm32f4xx_rcc.o(.text) refers to stm32f4xx_rcc.o(.data) for APBAHBPrescTable
    stm32f4xx_rng.o(.text) refers to stm32f4xx_rcc.o(.text) for RCC_AHB2PeriphResetCmd
    stm32f4xx_sdio.o(.text) refers to stm32f4xx_rcc.o(.text) for RCC_APB2PeriphResetCmd
    stm32f4xx_spi.o(.text) refers to stm32f4xx_rcc.o(.text) for RCC_APB2PeriphResetCmd
    stm32f4xx_syscfg.o(.text) refers to stm32f4xx_rcc.o(.text) for RCC_APB2PeriphResetCmd
    stm32f4xx_tim.o(.text) refers to stm32f4xx_rcc.o(.text) for RCC_APB2PeriphResetCmd
    stm32f4xx_usart.o(.text) refers to stm32f4xx_rcc.o(.text) for RCC_APB2PeriphResetCmd
    stm32f4xx_wwdg.o(.text) refers to stm32f4xx_rcc.o(.text) for RCC_APB1PeriphResetCmd
    usbd_audio_core.o(.text) refers to usb_dcd.o(.text) for DCD_EP_Open
    usbd_audio_core.o(.text) refers to usbd_ioreq.o(.text) for USBD_CtlPrepareRx
    usbd_audio_core.o(.text) refers to usbd_req.o(.text) for USBD_CtlError
    usbd_audio_core.o(.text) refers to usbd_audio_out_if.o(.data) for AUDIO_OUT_fops
    usbd_audio_core.o(.text) refers to usbd_audio_core.o(.bss) for IsocOutBuff
    usbd_audio_core.o(.text) refers to usbd_audio_core.o(.data) for AudioCtlCmd
    usbd_audio_core.o(.data) refers to usbd_audio_core.o(.bss) for IsocOutBuff
    usbd_audio_core.o(.data) refers to usbd_audio_core.o(.text) for usbd_audio_Init
    usbd_audio_out_if.o(.text) refers to stm32f4_discovery_audio_codec.o(.text) for EVAL_AUDIO_Init
    usbd_audio_out_if.o(.text) refers to usbd_audio_out_if.o(.data) for Initialized
    usbd_audio_out_if.o(.data) refers to usbd_audio_out_if.o(.text) for Init
    usbd_core.o(.text) refers to usb_bsp.o(.text) for USB_OTG_BSP_Init
    usbd_core.o(.text) refers to usb_dcd.o(.text) for DCD_Init
    usbd_core.o(.text) refers to usbd_req.o(.text) for USBD_ParseSetupRequest
    usbd_core.o(.text) refers to usbd_ioreq.o(.text) for USBD_CtlContinueRx
    usbd_core.o(.data) refers to usbd_core.o(.text) for USBD_DataOutStage
    usbd_ioreq.o(.text) refers to usb_dcd.o(.text) for DCD_EP_Tx
    usbd_ioreq.o(.text) refers to usb_core.o(.text) for USB_OTG_EP0_OutStart
    usbd_req.o(.text) refers to usb_dcd.o(.text) for DCD_EP_Stall
    usbd_req.o(.text) refers to usb_core.o(.text) for USB_OTG_EP0_OutStart
    usbd_req.o(.text) refers to usbd_ioreq.o(.text) for USBD_CtlSendStatus
    usbd_req.o(.text) refers to usbd_core.o(.text) for USBD_SetCfg
    usbd_req.o(.text) refers to usbd_req.o(.data) for USBD_cfg_status
    usb_core.o(.text) refers to usb_bsp.o(.text) for USB_OTG_BSP_uDelay
    usb_dcd.o(.text) refers to usb_core.o(.text) for USB_OTG_SelectCore
    usb_dcd.o(.text) refers to usb_bsp.o(.text) for USB_OTG_BSP_mDelay
    usb_dcd_int.o(.text) refers to usb_core.o(.text) for USB_OTG_EP0Activate
    usb_dcd_int.o(.text) refers to usbd_core.o(.data) for USBD_DCD_INT_fops
    main.o(.text) refers to usbd_core.o(.text) for USBD_Init
    main.o(.text) refers to usbd_usr.o(.data) for USR_cb
    main.o(.text) refers to usbd_audio_core.o(.data) for AUDIO_cb
    main.o(.text) refers to usbd_desc.o(.data) for USR_desc
    main.o(.text) refers to main.o(.bss) for USB_OTG_dev
    main.o(.text) refers to main.o(.data) for TimingDelay
    stm32f4xx_it.o(.text) refers to system_stm32f4xx.o(.text) for SystemInit
    stm32f4xx_it.o(.text) refers to usb_core.o(.text) for USB_OTG_UngateClock
    stm32f4xx_it.o(.text) refers to stm32f4xx_exti.o(.text) for EXTI_ClearITPendingBit
    stm32f4xx_it.o(.text) refers to usb_dcd_int.o(.text) for USBD_OTG_ISR_Handler
    stm32f4xx_it.o(.text) refers to main.o(.bss) for USB_OTG_dev
    usb_bsp.o(.text) refers to stm32f4xx_rcc.o(.text) for RCC_AHB1PeriphClockCmd
    usb_bsp.o(.text) refers to stm32f4xx_gpio.o(.text) for GPIO_Init
    usb_bsp.o(.text) refers to stm32f4xx_exti.o(.text) for EXTI_ClearITPendingBit
    usb_bsp.o(.text) refers to misc.o(.text) for NVIC_PriorityGroupConfig
    usbd_desc.o(.text) refers to usbd_req.o(.text) for USBD_GetString
    usbd_desc.o(.text) refers to usbd_desc.o(.data) for USBD_DeviceDesc
    usbd_desc.o(.text) refers to usbd_req.o(.bss) for USBD_StrDesc
    usbd_desc.o(.data) refers to usbd_desc.o(.text) for USBD_USR_DeviceDescriptor
    usbd_usr.o(.text) refers to system_stm32f4xx.o(.data) for SystemCoreClock
    usbd_usr.o(.data) refers to usbd_usr.o(.text) for USBD_USR_Init
    stm32f4_discovery.o(.text) refers to stm32f4xx_rcc.o(.text) for RCC_AHB1PeriphClockCmd
    stm32f4_discovery.o(.text) refers to stm32f4xx_gpio.o(.text) for GPIO_Init
    stm32f4_discovery.o(.text) refers to stm32f4xx_syscfg.o(.text) for SYSCFG_EXTILineConfig
    stm32f4_discovery.o(.text) refers to stm32f4xx_exti.o(.text) for EXTI_Init
    stm32f4_discovery.o(.text) refers to misc.o(.text) for NVIC_Init
    stm32f4_discovery.o(.text) refers to stm32f4_discovery.o(.constdata) for GPIO_CLK
    stm32f4_discovery.o(.text) refers to stm32f4_discovery.o(.data) for GPIO_PORT
    stm32f4_discovery_audio_codec.o(.text) refers to misc.o(.text) for NVIC_Init
    stm32f4_discovery_audio_codec.o(.text) refers to stm32f4xx_spi.o(.text) for SPI_I2S_ITConfig
    stm32f4_discovery_audio_codec.o(.text) refers to stm32f4xx_rcc.o(.text) for RCC_APB1PeriphClockCmd
    stm32f4_discovery_audio_codec.o(.text) refers to stm32f4xx_dac.o(.text) for DAC_Init
    stm32f4_discovery_audio_codec.o(.text) refers to stm32f4xx_i2c.o(.text) for I2C_GetFlagStatus
    stm32f4_discovery_audio_codec.o(.text) refers to stm32f4_discovery_audio_codec.o(.data) for CurrAudioInterface
    stm32f4_discovery_audio_codec.o(.text) refers to stm32f4xx_gpio.o(.text) for GPIO_WriteBit
    stm32f4_discovery_audio_codec.o(.text) refers to stm32f4xx_dma.o(.text) for DMA_Cmd
    stm32f4_discovery_audio_codec.o(.text) refers to stm32f4_discovery.o(.text) for STM_EVAL_LEDToggle
    stm32f4_discovery_audio_codec.o(.text) refers to stm32f4_discovery_audio_codec.o(.bss) for DMA_InitStructure
    __main.o(!!!main) refers to rtentry.o(.ARM.Collect$$rtentry$$00000000) for __rt_entry
    rtentry.o(.ARM.Collect$$rtentry$$00000000) refers (Special) to rtentry2.o(.ARM.Collect$$rtentry$$0000000A) for __rt_entry_li
    rtentry.o(.ARM.Collect$$rtentry$$00000000) refers (Special) to rtentry2.o(.ARM.Collect$$rtentry$$0000000D) for __rt_entry_main
    rtentry.o(.ARM.Collect$$rtentry$$00000000) refers (Special) to rtentry2.o(.ARM.Collect$$rtentry$$0000000C) for __rt_entry_postli_1
    rtentry.o(.ARM.Collect$$rtentry$$00000000) refers (Special) to rtentry2.o(.ARM.Collect$$rtentry$$00000009) for __rt_entry_postsh_1
    rtentry.o(.ARM.Collect$$rtentry$$00000000) refers (Special) to rtentry2.o(.ARM.Collect$$rtentry$$00000002) for __rt_entry_presh_1
    rtentry.o(.ARM.Collect$$rtentry$$00000000) refers (Special) to rtentry4.o(.ARM.Collect$$rtentry$$00000004) for __rt_entry_sh
    rtentry2.o(.ARM.Collect$$rtentry$$00000008) refers to boardinit2.o(.text) for _platform_post_stackheap_init
    rtentry2.o(.ARM.Collect$$rtentry$$0000000A) refers to libinit.o(.ARM.Collect$$libinit$$00000000) for __rt_lib_init
    rtentry2.o(.ARM.Collect$$rtentry$$0000000B) refers to boardinit3.o(.text) for _platform_post_lib_init
    rtentry2.o(.ARM.Collect$$rtentry$$0000000D) refers to main.o(.text) for main
    rtentry2.o(.ARM.Collect$$rtentry$$0000000D) refers to exit.o(.text) for exit
    rtentry2.o(.ARM.exidx) refers to rtentry2.o(.ARM.Collect$$rtentry$$00000001) for .ARM.Collect$$rtentry$$00000001
    rtentry2.o(.ARM.exidx) refers to rtentry2.o(.ARM.Collect$$rtentry$$00000008) for .ARM.Collect$$rtentry$$00000008
    rtentry2.o(.ARM.exidx) refers to rtentry2.o(.ARM.Collect$$rtentry$$0000000A) for .ARM.Collect$$rtentry$$0000000A
    rtentry2.o(.ARM.exidx) refers to rtentry2.o(.ARM.Collect$$rtentry$$0000000B) for .ARM.Collect$$rtentry$$0000000B
    rtentry2.o(.ARM.exidx) refers to rtentry2.o(.ARM.Collect$$rtentry$$0000000D) for .ARM.Collect$$rtentry$$0000000D
    rtentry4.o(.ARM.Collect$$rtentry$$00000004) refers to sys_stackheap_outer.o(.text) for __user_setup_stackheap
    rtentry4.o(.ARM.exidx) refers to rtentry4.o(.ARM.Collect$$rtentry$$00000004) for .ARM.Collect$$rtentry$$00000004
    sys_stackheap_outer.o(.text) refers to libspace.o(.text) for __user_perproc_libspace
    sys_stackheap_outer.o(.text) refers to startup_stm32f40_41xxx.o(.text) for __user_initial_stackheap
    exit.o(.text) refers to rtexit.o(.ARM.Collect$$rtexit$$00000000) for __rt_exit
    libinit.o(.ARM.Collect$$libinit$$00000000) refers (Special) to libinit2.o(.ARM.Collect$$libinit$$0000002C) for __rt_lib_init_alloca_1
    libinit.o(.ARM.Collect$$libinit$$00000000) refers (Special) to libinit2.o(.ARM.Collect$$libinit$$0000002A) for __rt_lib_init_argv_1
    libinit.o(.ARM.Collect$$libinit$$00000000) refers (Special) to libinit2.o(.ARM.Collect$$libinit$$00000019) for __rt_lib_init_atexit_1
    libinit.o(.ARM.Collect$$libinit$$00000000) refers (Special) to libinit2.o(.ARM.Collect$$libinit$$0000001F) for __rt_lib_init_clock_1
    libinit.o(.ARM.Collect$$libinit$$00000000) refers (Special) to libinit2.o(.ARM.Collect$$libinit$$00000030) for __rt_lib_init_cpp_1
    libinit.o(.ARM.Collect$$libinit$$00000000) refers (Special) to libinit2.o(.ARM.Collect$$libinit$$0000002E) for __rt_lib_init_exceptions_1
    libinit.o(.ARM.Collect$$libinit$$00000000) refers (Special) to libinit2.o(.ARM.Collect$$libinit$$00000002) for __rt_lib_init_fp_1
    libinit.o(.ARM.Collect$$libinit$$00000000) refers (Special) to libinit2.o(.ARM.Collect$$libinit$$0000001D) for __rt_lib_init_fp_trap_1
    libinit.o(.ARM.Collect$$libinit$$00000000) refers (Special) to libinit2.o(.ARM.Collect$$libinit$$00000021) for __rt_lib_init_getenv_1
    libinit.o(.ARM.Collect$$libinit$$00000000) refers (Special) to libinit2.o(.ARM.Collect$$libinit$$00000008) for __rt_lib_init_heap_1
    libinit.o(.ARM.Collect$$libinit$$00000000) refers (Special) to libinit2.o(.ARM.Collect$$libinit$$0000000F) for __rt_lib_init_lc_collate_1
    libinit.o(.ARM.Collect$$libinit$$00000000) refers (Special) to libinit2.o(.ARM.Collect$$libinit$$00000011) for __rt_lib_init_lc_ctype_1
    libinit.o(.ARM.Collect$$libinit$$00000000) refers (Special) to libinit2.o(.ARM.Collect$$libinit$$00000013) for __rt_lib_init_lc_monetary_1
    libinit.o(.ARM.Collect$$libinit$$00000000) refers (Special) to libinit2.o(.ARM.Collect$$libinit$$00000015) for __rt_lib_init_lc_numeric_1
    libinit.o(.ARM.Collect$$libinit$$00000000) refers (Special) to libinit2.o(.ARM.Collect$$libinit$$00000017) for __rt_lib_init_lc_time_1
    libinit.o(.ARM.Collect$$libinit$$00000000) refers (Special) to libinit2.o(.ARM.Collect$$libinit$$0000000C) for __rt_lib_init_rand_1
    libinit.o(.ARM.Collect$$libinit$$00000000) refers (Special) to libinit2.o(.ARM.Collect$$libinit$$00000031) for __rt_lib_init_return
    libinit.o(.ARM.Collect$$libinit$$00000000) refers (Special) to libinit2.o(.ARM.Collect$$libinit$$0000001B) for __rt_lib_init_signal_1
    libinit.o(.ARM.Collect$$libinit$$00000000) refers (Special) to libinit2.o(.ARM.Collect$$libinit$$00000023) for __rt_lib_init_stdio_1
    libinit.o(.ARM.Collect$$libinit$$00000000) refers (Special) to libinit2.o(.ARM.Collect$$libinit$$0000000A) for __rt_lib_init_user_alloc_1
    libspace.o(.text) refers to libspace.o(.bss) for __libspace_start
    rtexit.o(.ARM.Collect$$rtexit$$00000000) refers (Special) to rtexit2.o(.ARM.Collect$$rtexit$$00000004) for __rt_exit_exit
    rtexit.o(.ARM.Collect$$rtexit$$00000000) refers (Special) to rtexit2.o(.ARM.Collect$$rtexit$$00000003) for __rt_exit_ls
    rtexit.o(.ARM.Collect$$rtexit$$00000000) refers (Special) to rtexit2.o(.ARM.Collect$$rtexit$$00000002) for __rt_exit_prels_1
    rtexit.o(.ARM.exidx) refers (Special) to rtexit2.o(.ARM.Collect$$rtexit$$00000004) for __rt_exit_exit
    rtexit.o(.ARM.exidx) refers (Special) to rtexit2.o(.ARM.Collect$$rtexit$$00000003) for __rt_exit_ls
    rtexit.o(.ARM.exidx) refers (Special) to rtexit2.o(.ARM.Collect$$rtexit$$00000002) for __rt_exit_prels_1
    rtexit.o(.ARM.exidx) refers to rtexit.o(.ARM.Collect$$rtexit$$00000000) for .ARM.Collect$$rtexit$$00000000
    libinit2.o(.ARM.Collect$$libinit$$0000000E) refers to libinit2.o(.ARM.Collect$$libinit$$0000000D) for .ARM.Collect$$libinit$$0000000D
    libinit2.o(.ARM.Collect$$libinit$$00000010) refers to libinit2.o(.ARM.Collect$$libinit$$0000000D) for .ARM.Collect$$libinit$$0000000D
    libinit2.o(.ARM.Collect$$libinit$$00000012) refers to libinit2.o(.ARM.Collect$$libinit$$0000000D) for .ARM.Collect$$libinit$$0000000D
    libinit2.o(.ARM.Collect$$libinit$$00000014) refers to libinit2.o(.ARM.Collect$$libinit$$0000000D) for .ARM.Collect$$libinit$$0000000D
    libinit2.o(.ARM.Collect$$libinit$$00000016) refers to libinit2.o(.ARM.Collect$$libinit$$0000000D) for .ARM.Collect$$libinit$$0000000D
    libinit2.o(.ARM.Collect$$libinit$$00000024) refers to argv_veneer.o(.emb_text) for __ARM_argv_veneer
    libinit2.o(.ARM.Collect$$libinit$$00000025) refers to argv_veneer.o(.emb_text) for __ARM_argv_veneer
    rtexit2.o(.ARM.Collect$$rtexit$$00000003) refers to libshutdown.o(.ARM.Collect$$libshutdown$$00000000) for __rt_lib_shutdown
    rtexit2.o(.ARM.Collect$$rtexit$$00000004) refers to sys_exit.o(.text) for _sys_exit
    rtexit2.o(.ARM.exidx) refers to rtexit2.o(.ARM.Collect$$rtexit$$00000001) for .ARM.Collect$$rtexit$$00000001
    rtexit2.o(.ARM.exidx) refers to rtexit2.o(.ARM.Collect$$rtexit$$00000003) for .ARM.Collect$$rtexit$$00000003
    rtexit2.o(.ARM.exidx) refers to rtexit2.o(.ARM.Collect$$rtexit$$00000004) for .ARM.Collect$$rtexit$$00000004
    argv_veneer.o(.emb_text) refers to no_argv.o(.text) for __ARM_get_argv
    sys_exit.o(.text) refers (Special) to use_no_semi.o(.text) for __I$use$semihosting
    sys_exit.o(.text) refers (Special) to indicate_semi.o(.text) for __semihosting_library_function
    _get_argv_nomalloc.o(.text) refers (Special) to hrguard.o(.text) for __heap_region$guard
    _get_argv_nomalloc.o(.text) refers to defsig_rtmem_outer.o(.text) for __rt_SIGRTMEM
    _get_argv_nomalloc.o(.text) refers to sys_command.o(.text) for _sys_command_string
    libshutdown.o(.ARM.Collect$$libshutdown$$00000000) refers (Special) to libshutdown2.o(.ARM.Collect$$libshutdown$$00000006) for __rt_lib_shutdown_fp_trap_1
    libshutdown.o(.ARM.Collect$$libshutdown$$00000000) refers (Special) to libshutdown2.o(.ARM.Collect$$libshutdown$$0000000E) for __rt_lib_shutdown_heap_1
    libshutdown.o(.ARM.Collect$$libshutdown$$00000000) refers (Special) to libshutdown2.o(.ARM.Collect$$libshutdown$$0000000F) for __rt_lib_shutdown_return
    libshutdown.o(.ARM.Collect$$libshutdown$$00000000) refers (Special) to libshutdown2.o(.ARM.Collect$$libshutdown$$00000009) for __rt_lib_shutdown_signal_1
    libshutdown.o(.ARM.Collect$$libshutdown$$00000000) refers (Special) to libshutdown2.o(.ARM.Collect$$libshutdown$$00000003) for __rt_lib_shutdown_stdio_1
    libshutdown.o(.ARM.Collect$$libshutdown$$00000000) refers (Special) to libshutdown2.o(.ARM.Collect$$libshutdown$$0000000B) for __rt_lib_shutdown_user_alloc_1
    sys_command.o(.text) refers (Special) to use_no_semi.o(.text) for __I$use$semihosting
    sys_command.o(.text) refers (Special) to indicate_semi.o(.text) for __semihosting_library_function
    defsig_rtmem_outer.o(.text) refers to defsig_rtmem_inner.o(.text) for __rt_SIGRTMEM_inner
    defsig_rtmem_outer.o(.text) refers to defsig_exit.o(.text) for __sig_exit
    defsig_rtmem_formal.o(.text) refers to rt_raise.o(.text) for __rt_raise
    rt_raise.o(.text) refers to __raise.o(.text) for __raise
    rt_raise.o(.text) refers to sys_exit.o(.text) for _sys_exit
    defsig_exit.o(.text) refers to sys_exit.o(.text) for _sys_exit
    defsig_rtmem_inner.o(.text) refers to defsig_general.o(.text) for __default_signal_display
    __raise.o(.text) refers to defsig.o(CL$$defsig) for __default_signal_handler
    defsig_general.o(.text) refers to sys_wrch.o(.text) for _ttywrch
    sys_wrch.o(.text) refers (Special) to use_no_semi.o(.text) for __I$use$semihosting
    sys_wrch.o(.text) refers (Special) to indicate_semi.o(.text) for __semihosting_library_function
    defsig.o(CL$$defsig) refers to defsig_rtmem_inner.o(.text) for __rt_SIGRTMEM_inner
    defsig_abrt_inner.o(.text) refers to defsig_general.o(.text) for __default_signal_display
    defsig_fpe_inner.o(.text) refers to defsig_general.o(.text) for __default_signal_display
    defsig_rtred_inner.o(.text) refers to defsig_general.o(.text) for __default_signal_display
    defsig_stak_inner.o(.text) refers to defsig_general.o(.text) for __default_signal_display
    defsig_pvfn_inner.o(.text) refers to defsig_general.o(.text) for __default_signal_display
    defsig_cppl_inner.o(.text) refers to defsig_general.o(.text) for __default_signal_display
    defsig_segv_inner.o(.text) refers to defsig_general.o(.text) for __default_signal_display
    defsig_other.o(.text) refers to defsig_general.o(.text) for __default_signal_display


==============================================================================

Removing Unused input sections from the image.

    Removing system_stm32f4xx.o(.rev16_text), (4 bytes).
    Removing system_stm32f4xx.o(.revsh_text), (4 bytes).
    Removing misc.o(.rev16_text), (4 bytes).
    Removing misc.o(.revsh_text), (4 bytes).
    Removing stm32f4xx_adc.o(.rev16_text), (4 bytes).
    Removing stm32f4xx_adc.o(.revsh_text), (4 bytes).
    Removing stm32f4xx_adc.o(.text), (1136 bytes).
    Removing stm32f4xx_can.o(.rev16_text), (4 bytes).
    Removing stm32f4xx_can.o(.revsh_text), (4 bytes).
    Removing stm32f4xx_can.o(.text), (2540 bytes).
    Removing stm32f4xx_crc.o(.rev16_text), (4 bytes).
    Removing stm32f4xx_crc.o(.revsh_text), (4 bytes).
    Removing stm32f4xx_crc.o(.text), (72 bytes).
    Removing stm32f4xx_cryp.o(.rev16_text), (4 bytes).
    Removing stm32f4xx_cryp.o(.revsh_text), (4 bytes).
    Removing stm32f4xx_cryp.o(.text), (664 bytes).
    Removing stm32f4xx_cryp_aes.o(.rev16_text), (4 bytes).
    Removing stm32f4xx_cryp_aes.o(.revsh_text), (4 bytes).
    Removing stm32f4xx_cryp_aes.o(.text), (1524 bytes).
    Removing stm32f4xx_cryp_des.o(.rev16_text), (4 bytes).
    Removing stm32f4xx_cryp_des.o(.revsh_text), (4 bytes).
    Removing stm32f4xx_cryp_des.o(.text), (468 bytes).
    Removing stm32f4xx_cryp_tdes.o(.rev16_text), (4 bytes).
    Removing stm32f4xx_cryp_tdes.o(.revsh_text), (4 bytes).
    Removing stm32f4xx_cryp_tdes.o(.text), (532 bytes).
    Removing stm32f4xx_dac.o(.rev16_text), (4 bytes).
    Removing stm32f4xx_dac.o(.revsh_text), (4 bytes).
    Removing stm32f4xx_dbgmcu.o(.rev16_text), (4 bytes).
    Removing stm32f4xx_dbgmcu.o(.revsh_text), (4 bytes).
    Removing stm32f4xx_dbgmcu.o(.text), (100 bytes).
    Removing stm32f4xx_dcmi.o(.rev16_text), (4 bytes).
    Removing stm32f4xx_dcmi.o(.revsh_text), (4 bytes).
    Removing stm32f4xx_dcmi.o(.text), (396 bytes).
    Removing stm32f4xx_dma.o(.rev16_text), (4 bytes).
    Removing stm32f4xx_dma.o(.revsh_text), (4 bytes).
    Removing stm32f4xx_exti.o(.rev16_text), (4 bytes).
    Removing stm32f4xx_exti.o(.revsh_text), (4 bytes).
    Removing stm32f4xx_flash.o(.rev16_text), (4 bytes).
    Removing stm32f4xx_flash.o(.revsh_text), (4 bytes).
    Removing stm32f4xx_flash.o(.text), (1224 bytes).
    Removing stm32f4xx_fsmc.o(.rev16_text), (4 bytes).
    Removing stm32f4xx_fsmc.o(.revsh_text), (4 bytes).
    Removing stm32f4xx_fsmc.o(.text), (1564 bytes).
    Removing stm32f4xx_gpio.o(.rev16_text), (4 bytes).
    Removing stm32f4xx_gpio.o(.revsh_text), (4 bytes).
    Removing stm32f4xx_hash.o(.rev16_text), (4 bytes).
    Removing stm32f4xx_hash.o(.revsh_text), (4 bytes).
    Removing stm32f4xx_hash.o(.text), (500 bytes).
    Removing stm32f4xx_hash_md5.o(.rev16_text), (4 bytes).
    Removing stm32f4xx_hash_md5.o(.revsh_text), (4 bytes).
    Removing stm32f4xx_hash_md5.o(.text), (534 bytes).
    Removing stm32f4xx_hash_sha1.o(.rev16_text), (4 bytes).
    Removing stm32f4xx_hash_sha1.o(.revsh_text), (4 bytes).
    Removing stm32f4xx_hash_sha1.o(.text), (548 bytes).
    Removing stm32f4xx_i2c.o(.rev16_text), (4 bytes).
    Removing stm32f4xx_i2c.o(.revsh_text), (4 bytes).
    Removing stm32f4xx_iwdg.o(.rev16_text), (4 bytes).
    Removing stm32f4xx_iwdg.o(.revsh_text), (4 bytes).
    Removing stm32f4xx_iwdg.o(.text), (64 bytes).
    Removing stm32f4xx_pwr.o(.rev16_text), (4 bytes).
    Removing stm32f4xx_pwr.o(.revsh_text), (4 bytes).
    Removing stm32f4xx_pwr.o(.text), (252 bytes).
    Removing stm32f4xx_rcc.o(.rev16_text), (4 bytes).
    Removing stm32f4xx_rcc.o(.revsh_text), (4 bytes).
    Removing stm32f4xx_rng.o(.rev16_text), (4 bytes).
    Removing stm32f4xx_rng.o(.revsh_text), (4 bytes).
    Removing stm32f4xx_rng.o(.text), (160 bytes).
    Removing stm32f4xx_rtc.o(.rev16_text), (4 bytes).
    Removing stm32f4xx_rtc.o(.revsh_text), (4 bytes).
    Removing stm32f4xx_rtc.o(.text), (3376 bytes).
    Removing stm32f4xx_sdio.o(.rev16_text), (4 bytes).
    Removing stm32f4xx_sdio.o(.revsh_text), (4 bytes).
    Removing stm32f4xx_sdio.o(.text), (484 bytes).
    Removing stm32f4xx_spi.o(.rev16_text), (4 bytes).
    Removing stm32f4xx_spi.o(.revsh_text), (4 bytes).
    Removing stm32f4xx_syscfg.o(.rev16_text), (4 bytes).
    Removing stm32f4xx_syscfg.o(.revsh_text), (4 bytes).
    Removing stm32f4xx_tim.o(.rev16_text), (4 bytes).
    Removing stm32f4xx_tim.o(.revsh_text), (4 bytes).
    Removing stm32f4xx_tim.o(.text), (3234 bytes).
    Removing stm32f4xx_usart.o(.rev16_text), (4 bytes).
    Removing stm32f4xx_usart.o(.revsh_text), (4 bytes).
    Removing stm32f4xx_usart.o(.text), (1050 bytes).
    Removing stm32f4xx_wwdg.o(.rev16_text), (4 bytes).
    Removing stm32f4xx_wwdg.o(.revsh_text), (4 bytes).
    Removing stm32f4xx_wwdg.o(.text), (144 bytes).
    Removing usbd_audio_core.o(.rev16_text), (4 bytes).
    Removing usbd_audio_core.o(.revsh_text), (4 bytes).
    Removing usbd_audio_out_if.o(.rev16_text), (4 bytes).
    Removing usbd_audio_out_if.o(.revsh_text), (4 bytes).
    Removing usbd_core.o(.rev16_text), (4 bytes).
    Removing usbd_core.o(.revsh_text), (4 bytes).
    Removing usbd_ioreq.o(.rev16_text), (4 bytes).
    Removing usbd_ioreq.o(.revsh_text), (4 bytes).
    Removing usbd_req.o(.rev16_text), (4 bytes).
    Removing usbd_req.o(.revsh_text), (4 bytes).
    Removing usb_core.o(.rev16_text), (4 bytes).
    Removing usb_core.o(.revsh_text), (4 bytes).
    Removing usb_dcd.o(.rev16_text), (4 bytes).
    Removing usb_dcd.o(.revsh_text), (4 bytes).
    Removing usb_dcd_int.o(.rev16_text), (4 bytes).
    Removing usb_dcd_int.o(.revsh_text), (4 bytes).
    Removing main.o(.rev16_text), (4 bytes).
    Removing main.o(.revsh_text), (4 bytes).
    Removing stm32f4xx_it.o(.rev16_text), (4 bytes).
    Removing stm32f4xx_it.o(.revsh_text), (4 bytes).
    Removing usb_bsp.o(.rev16_text), (4 bytes).
    Removing usb_bsp.o(.revsh_text), (4 bytes).
    Removing usbd_desc.o(.rev16_text), (4 bytes).
    Removing usbd_desc.o(.revsh_text), (4 bytes).
    Removing usbd_usr.o(.rev16_text), (4 bytes).
    Removing usbd_usr.o(.revsh_text), (4 bytes).
    Removing stm32f4_discovery.o(.rev16_text), (4 bytes).
    Removing stm32f4_discovery.o(.revsh_text), (4 bytes).
    Removing stm32f4_discovery_audio_codec.o(.rev16_text), (4 bytes).
    Removing stm32f4_discovery_audio_codec.o(.revsh_text), (4 bytes).

116 unused section(s) (total 20942 bytes) removed from the image.

==============================================================================

Image Symbol Table

    Local Symbols

    Symbol Name                              Value     Ov Type        Size  Object(Section)

    ../clib/angel/boardlib.s                 0x00000000   Number         0  boardinit2.o ABSOLUTE
    ../clib/angel/boardlib.s                 0x00000000   Number         0  boardinit3.o ABSOLUTE
    ../clib/angel/boardlib.s                 0x00000000   Number         0  boardinit1.o ABSOLUTE
    ../clib/angel/boardlib.s                 0x00000000   Number         0  boardshut.o ABSOLUTE
    ../clib/angel/dczerorl2.s                0x00000000   Number         0  __dczerorl2.o ABSOLUTE
    ../clib/angel/handlers.s                 0x00000000   Number         0  __scatter_zi.o ABSOLUTE
    ../clib/angel/kernel.s                   0x00000000   Number         0  rtexit.o ABSOLUTE
    ../clib/angel/kernel.s                   0x00000000   Number         0  rtexit2.o ABSOLUTE
    ../clib/angel/kernel.s                   0x00000000   Number         0  rtentry.o ABSOLUTE
    ../clib/angel/kernel.s                   0x00000000   Number         0  rtentry4.o ABSOLUTE
    ../clib/angel/kernel.s                   0x00000000   Number         0  rtentry2.o ABSOLUTE
    ../clib/angel/rt.s                       0x00000000   Number         0  rt_raise.o ABSOLUTE
    ../clib/angel/scatter.s                  0x00000000   Number         0  __scatter.o ABSOLUTE
    ../clib/angel/startup.s                  0x00000000   Number         0  __main.o ABSOLUTE
    ../clib/angel/sys.s                      0x00000000   Number         0  libspace.o ABSOLUTE
    ../clib/angel/sys.s                      0x00000000   Number         0  indicate_semi.o ABSOLUTE
    ../clib/angel/sys.s                      0x00000000   Number         0  sys_stackheap_outer.o ABSOLUTE
    ../clib/angel/sys.s                      0x00000000   Number         0  use_no_semi.o ABSOLUTE
    ../clib/angel/sysapp.c                   0x00000000   Number         0  sys_command.o ABSOLUTE
    ../clib/angel/sysapp.c                   0x00000000   Number         0  sys_exit.o ABSOLUTE
    ../clib/angel/sysapp.c                   0x00000000   Number         0  sys_wrch.o ABSOLUTE
    ../clib/armsys.c                         0x00000000   Number         0  argv_veneer.o ABSOLUTE
    ../clib/armsys.c                         0x00000000   Number         0  no_argv.o ABSOLUTE
    ../clib/armsys.c                         0x00000000   Number         0  _get_argv_nomalloc.o ABSOLUTE
    ../clib/armsys.c                         0x00000000   Number         0  argv_veneer.o ABSOLUTE
    ../clib/heapalloc.c                      0x00000000   Number         0  hrguard.o ABSOLUTE
    ../clib/heapaux.c                        0x00000000   Number         0  heapauxi.o ABSOLUTE
    ../clib/libinit.s                        0x00000000   Number         0  libinit.o ABSOLUTE
    ../clib/libinit.s                        0x00000000   Number         0  libshutdown.o ABSOLUTE
    ../clib/libinit.s                        0x00000000   Number         0  libinit2.o ABSOLUTE
    ../clib/libinit.s                        0x00000000   Number         0  libshutdown2.o ABSOLUTE
    ../clib/signal.c                         0x00000000   Number         0  defsig_rtmem_formal.o ABSOLUTE
    ../clib/signal.c                         0x00000000   Number         0  defsig_abrt_inner.o ABSOLUTE
    ../clib/signal.c                         0x00000000   Number         0  defsig_other.o ABSOLUTE
    ../clib/signal.c                         0x00000000   Number         0  defsig_exit.o ABSOLUTE
    ../clib/signal.c                         0x00000000   Number         0  defsig_rtmem_outer.o ABSOLUTE
    ../clib/signal.c                         0x00000000   Number         0  defsig_rtmem_inner.o ABSOLUTE
    ../clib/signal.c                         0x00000000   Number         0  __raise.o ABSOLUTE
    ../clib/signal.c                         0x00000000   Number         0  defsig_general.o ABSOLUTE
    ../clib/signal.c                         0x00000000   Number         0  defsig_segv_inner.o ABSOLUTE
    ../clib/signal.c                         0x00000000   Number         0  defsig_fpe_inner.o ABSOLUTE
    ../clib/signal.c                         0x00000000   Number         0  defsig_rtred_inner.o ABSOLUTE
    ../clib/signal.c                         0x00000000   Number         0  defsig_stak_inner.o ABSOLUTE
    ../clib/signal.c                         0x00000000   Number         0  defsig_pvfn_inner.o ABSOLUTE
    ../clib/signal.c                         0x00000000   Number         0  defsig_cppl_inner.o ABSOLUTE
    ../clib/signal.s                         0x00000000   Number         0  defsig.o ABSOLUTE
    ../clib/stdlib.c                         0x00000000   Number         0  exit.o ABSOLUTE
    ../fplib/fpinit.s                        0x00000000   Number         0  fpinit.o ABSOLUTE
    ..\App\main.c                            0x00000000   Number         0  main.o ABSOLUTE
    ..\App\stm32f4xx_it.c                    0x00000000   Number         0  stm32f4xx_it.o ABSOLUTE
    ..\App\system_stm32f4xx.c                0x00000000   Number         0  system_stm32f4xx.o ABSOLUTE
    ..\App\usb_bsp.c                         0x00000000   Number         0  usb_bsp.o ABSOLUTE
    ..\App\usbd_desc.c                       0x00000000   Number         0  usbd_desc.o ABSOLUTE
    ..\App\usbd_usr.c                        0x00000000   Number         0  usbd_usr.o ABSOLUTE
    ..\STM32F4-Discovery\stm32f4_discovery.c 0x00000000   Number         0  stm32f4_discovery.o ABSOLUTE
    ..\STM32F4-Discovery\stm32f4_discovery_audio_codec.c 0x00000000   Number         0  stm32f4_discovery_audio_codec.o ABSOLUTE
    ..\STM32F4xx_StdPeriph_Driver\src\misc.c 0x00000000   Number         0  misc.o ABSOLUTE
    ..\STM32F4xx_StdPeriph_Driver\src\stm32f4xx_adc.c 0x00000000   Number         0  stm32f4xx_adc.o ABSOLUTE
    ..\STM32F4xx_StdPeriph_Driver\src\stm32f4xx_can.c 0x00000000   Number         0  stm32f4xx_can.o ABSOLUTE
    ..\STM32F4xx_StdPeriph_Driver\src\stm32f4xx_crc.c 0x00000000   Number         0  stm32f4xx_crc.o ABSOLUTE
    ..\STM32F4xx_StdPeriph_Driver\src\stm32f4xx_cryp.c 0x00000000   Number         0  stm32f4xx_cryp.o ABSOLUTE
    ..\STM32F4xx_StdPeriph_Driver\src\stm32f4xx_cryp_aes.c 0x00000000   Number         0  stm32f4xx_cryp_aes.o ABSOLUTE
    ..\STM32F4xx_StdPeriph_Driver\src\stm32f4xx_cryp_des.c 0x00000000   Number         0  stm32f4xx_cryp_des.o ABSOLUTE
    ..\STM32F4xx_StdPeriph_Driver\src\stm32f4xx_cryp_tdes.c 0x00000000   Number         0  stm32f4xx_cryp_tdes.o ABSOLUTE
    ..\STM32F4xx_StdPeriph_Driver\src\stm32f4xx_dac.c 0x00000000   Number         0  stm32f4xx_dac.o ABSOLUTE
    ..\STM32F4xx_StdPeriph_Driver\src\stm32f4xx_dbgmcu.c 0x00000000   Number         0  stm32f4xx_dbgmcu.o ABSOLUTE
    ..\STM32F4xx_StdPeriph_Driver\src\stm32f4xx_dcmi.c 0x00000000   Number         0  stm32f4xx_dcmi.o ABSOLUTE
    ..\STM32F4xx_StdPeriph_Driver\src\stm32f4xx_dma.c 0x00000000   Number         0  stm32f4xx_dma.o ABSOLUTE
    ..\STM32F4xx_StdPeriph_Driver\src\stm32f4xx_exti.c 0x00000000   Number         0  stm32f4xx_exti.o ABSOLUTE
    ..\STM32F4xx_StdPeriph_Driver\src\stm32f4xx_flash.c 0x00000000   Number         0  stm32f4xx_flash.o ABSOLUTE
    ..\STM32F4xx_StdPeriph_Driver\src\stm32f4xx_fsmc.c 0x00000000   Number         0  stm32f4xx_fsmc.o ABSOLUTE
    ..\STM32F4xx_StdPeriph_Driver\src\stm32f4xx_gpio.c 0x00000000   Number         0  stm32f4xx_gpio.o ABSOLUTE
    ..\STM32F4xx_StdPeriph_Driver\src\stm32f4xx_hash.c 0x00000000   Number         0  stm32f4xx_hash.o ABSOLUTE
    ..\STM32F4xx_StdPeriph_Driver\src\stm32f4xx_hash_md5.c 0x00000000   Number         0  stm32f4xx_hash_md5.o ABSOLUTE
    ..\STM32F4xx_StdPeriph_Driver\src\stm32f4xx_hash_sha1.c 0x00000000   Number         0  stm32f4xx_hash_sha1.o ABSOLUTE
    ..\STM32F4xx_StdPeriph_Driver\src\stm32f4xx_i2c.c 0x00000000   Number         0  stm32f4xx_i2c.o ABSOLUTE
    ..\STM32F4xx_StdPeriph_Driver\src\stm32f4xx_iwdg.c 0x00000000   Number         0  stm32f4xx_iwdg.o ABSOLUTE
    ..\STM32F4xx_StdPeriph_Driver\src\stm32f4xx_pwr.c 0x00000000   Number         0  stm32f4xx_pwr.o ABSOLUTE
    ..\STM32F4xx_StdPeriph_Driver\src\stm32f4xx_rcc.c 0x00000000   Number         0  stm32f4xx_rcc.o ABSOLUTE
    ..\STM32F4xx_StdPeriph_Driver\src\stm32f4xx_rng.c 0x00000000   Number         0  stm32f4xx_rng.o ABSOLUTE
    ..\STM32F4xx_StdPeriph_Driver\src\stm32f4xx_rtc.c 0x00000000   Number         0  stm32f4xx_rtc.o ABSOLUTE
    ..\STM32F4xx_StdPeriph_Driver\src\stm32f4xx_sdio.c 0x00000000   Number         0  stm32f4xx_sdio.o ABSOLUTE
    ..\STM32F4xx_StdPeriph_Driver\src\stm32f4xx_spi.c 0x00000000   Number         0  stm32f4xx_spi.o ABSOLUTE
    ..\STM32F4xx_StdPeriph_Driver\src\stm32f4xx_syscfg.c 0x00000000   Number         0  stm32f4xx_syscfg.o ABSOLUTE
    ..\STM32F4xx_StdPeriph_Driver\src\stm32f4xx_tim.c 0x00000000   Number         0  stm32f4xx_tim.o ABSOLUTE
    ..\STM32F4xx_StdPeriph_Driver\src\stm32f4xx_usart.c 0x00000000   Number         0  stm32f4xx_usart.o ABSOLUTE
    ..\STM32F4xx_StdPeriph_Driver\src\stm32f4xx_wwdg.c 0x00000000   Number         0  stm32f4xx_wwdg.o ABSOLUTE
    ..\STM32_USB_Device_Library\Class\audio\src\usbd_audio_core.c 0x00000000   Number         0  usbd_audio_core.o ABSOLUTE
    ..\STM32_USB_Device_Library\Class\audio\src\usbd_audio_out_if.c 0x00000000   Number         0  usbd_audio_out_if.o ABSOLUTE
    ..\STM32_USB_Device_Library\Core\src\usbd_core.c 0x00000000   Number         0  usbd_core.o ABSOLUTE
    ..\STM32_USB_Device_Library\Core\src\usbd_ioreq.c 0x00000000   Number         0  usbd_ioreq.o ABSOLUTE
    ..\STM32_USB_Device_Library\Core\src\usbd_req.c 0x00000000   Number         0  usbd_req.o ABSOLUTE
    ..\STM32_USB_OTG_Driver\src\usb_core.c   0x00000000   Number         0  usb_core.o ABSOLUTE
    ..\STM32_USB_OTG_Driver\src\usb_dcd.c    0x00000000   Number         0  usb_dcd.o ABSOLUTE
    ..\STM32_USB_OTG_Driver\src\usb_dcd_int.c 0x00000000   Number         0  usb_dcd_int.o ABSOLUTE
    ..\\App\\main.c                          0x00000000   Number         0  main.o ABSOLUTE
    ..\\App\\stm32f4xx_it.c                  0x00000000   Number         0  stm32f4xx_it.o ABSOLUTE
    ..\\App\\system_stm32f4xx.c              0x00000000   Number         0  system_stm32f4xx.o ABSOLUTE
    ..\\App\\usb_bsp.c                       0x00000000   Number         0  usb_bsp.o ABSOLUTE
    ..\\App\\usbd_desc.c                     0x00000000   Number         0  usbd_desc.o ABSOLUTE
    ..\\App\\usbd_usr.c                      0x00000000   Number         0  usbd_usr.o ABSOLUTE
    ..\\STM32F4-Discovery\\stm32f4_discovery.c 0x00000000   Number         0  stm32f4_discovery.o ABSOLUTE
    ..\\STM32F4-Discovery\\stm32f4_discovery_audio_codec.c 0x00000000   Number         0  stm32f4_discovery_audio_codec.o ABSOLUTE
    ..\\STM32F4xx_StdPeriph_Driver\\src\\misc.c 0x00000000   Number         0  misc.o ABSOLUTE
    ..\\STM32F4xx_StdPeriph_Driver\\src\\stm32f4xx_adc.c 0x00000000   Number         0  stm32f4xx_adc.o ABSOLUTE
    ..\\STM32F4xx_StdPeriph_Driver\\src\\stm32f4xx_can.c 0x00000000   Number         0  stm32f4xx_can.o ABSOLUTE
    ..\\STM32F4xx_StdPeriph_Driver\\src\\stm32f4xx_crc.c 0x00000000   Number         0  stm32f4xx_crc.o ABSOLUTE
    ..\\STM32F4xx_StdPeriph_Driver\\src\\stm32f4xx_cryp.c 0x00000000   Number         0  stm32f4xx_cryp.o ABSOLUTE
    ..\\STM32F4xx_StdPeriph_Driver\\src\\stm32f4xx_cryp_aes.c 0x00000000   Number         0  stm32f4xx_cryp_aes.o ABSOLUTE
    ..\\STM32F4xx_StdPeriph_Driver\\src\\stm32f4xx_cryp_des.c 0x00000000   Number         0  stm32f4xx_cryp_des.o ABSOLUTE
    ..\\STM32F4xx_StdPeriph_Driver\\src\\stm32f4xx_cryp_tdes.c 0x00000000   Number         0  stm32f4xx_cryp_tdes.o ABSOLUTE
    ..\\STM32F4xx_StdPeriph_Driver\\src\\stm32f4xx_dac.c 0x00000000   Number         0  stm32f4xx_dac.o ABSOLUTE
    ..\\STM32F4xx_StdPeriph_Driver\\src\\stm32f4xx_dbgmcu.c 0x00000000   Number         0  stm32f4xx_dbgmcu.o ABSOLUTE
    ..\\STM32F4xx_StdPeriph_Driver\\src\\stm32f4xx_dcmi.c 0x00000000   Number         0  stm32f4xx_dcmi.o ABSOLUTE
    ..\\STM32F4xx_StdPeriph_Driver\\src\\stm32f4xx_dma.c 0x00000000   Number         0  stm32f4xx_dma.o ABSOLUTE
    ..\\STM32F4xx_StdPeriph_Driver\\src\\stm32f4xx_exti.c 0x00000000   Number         0  stm32f4xx_exti.o ABSOLUTE
    ..\\STM32F4xx_StdPeriph_Driver\\src\\stm32f4xx_flash.c 0x00000000   Number         0  stm32f4xx_flash.o ABSOLUTE
    ..\\STM32F4xx_StdPeriph_Driver\\src\\stm32f4xx_fsmc.c 0x00000000   Number         0  stm32f4xx_fsmc.o ABSOLUTE
    ..\\STM32F4xx_StdPeriph_Driver\\src\\stm32f4xx_gpio.c 0x00000000   Number         0  stm32f4xx_gpio.o ABSOLUTE
    ..\\STM32F4xx_StdPeriph_Driver\\src\\stm32f4xx_hash.c 0x00000000   Number         0  stm32f4xx_hash.o ABSOLUTE
    ..\\STM32F4xx_StdPeriph_Driver\\src\\stm32f4xx_hash_md5.c 0x00000000   Number         0  stm32f4xx_hash_md5.o ABSOLUTE
    ..\\STM32F4xx_StdPeriph_Driver\\src\\stm32f4xx_hash_sha1.c 0x00000000   Number         0  stm32f4xx_hash_sha1.o ABSOLUTE
    ..\\STM32F4xx_StdPeriph_Driver\\src\\stm32f4xx_i2c.c 0x00000000   Number         0  stm32f4xx_i2c.o ABSOLUTE
    ..\\STM32F4xx_StdPeriph_Driver\\src\\stm32f4xx_iwdg.c 0x00000000   Number         0  stm32f4xx_iwdg.o ABSOLUTE
    ..\\STM32F4xx_StdPeriph_Driver\\src\\stm32f4xx_pwr.c 0x00000000   Number         0  stm32f4xx_pwr.o ABSOLUTE
    ..\\STM32F4xx_StdPeriph_Driver\\src\\stm32f4xx_rcc.c 0x00000000   Number         0  stm32f4xx_rcc.o ABSOLUTE
    ..\\STM32F4xx_StdPeriph_Driver\\src\\stm32f4xx_rng.c 0x00000000   Number         0  stm32f4xx_rng.o ABSOLUTE
    ..\\STM32F4xx_StdPeriph_Driver\\src\\stm32f4xx_rtc.c 0x00000000   Number         0  stm32f4xx_rtc.o ABSOLUTE
    ..\\STM32F4xx_StdPeriph_Driver\\src\\stm32f4xx_sdio.c 0x00000000   Number         0  stm32f4xx_sdio.o ABSOLUTE
    ..\\STM32F4xx_StdPeriph_Driver\\src\\stm32f4xx_spi.c 0x00000000   Number         0  stm32f4xx_spi.o ABSOLUTE
    ..\\STM32F4xx_StdPeriph_Driver\\src\\stm32f4xx_syscfg.c 0x00000000   Number         0  stm32f4xx_syscfg.o ABSOLUTE
    ..\\STM32F4xx_StdPeriph_Driver\\src\\stm32f4xx_tim.c 0x00000000   Number         0  stm32f4xx_tim.o ABSOLUTE
    ..\\STM32F4xx_StdPeriph_Driver\\src\\stm32f4xx_usart.c 0x00000000   Number         0  stm32f4xx_usart.o ABSOLUTE
    ..\\STM32F4xx_StdPeriph_Driver\\src\\stm32f4xx_wwdg.c 0x00000000   Number         0  stm32f4xx_wwdg.o ABSOLUTE
    ..\\STM32_USB_Device_Library\\Class\\audio\\src\\usbd_audio_core.c 0x00000000   Number         0  usbd_audio_core.o ABSOLUTE
    ..\\STM32_USB_Device_Library\\Class\\audio\\src\\usbd_audio_out_if.c 0x00000000   Number         0  usbd_audio_out_if.o ABSOLUTE
    ..\\STM32_USB_Device_Library\\Core\\src\\usbd_core.c 0x00000000   Number         0  usbd_core.o ABSOLUTE
    ..\\STM32_USB_Device_Library\\Core\\src\\usbd_ioreq.c 0x00000000   Number         0  usbd_ioreq.o ABSOLUTE
    ..\\STM32_USB_Device_Library\\Core\\src\\usbd_req.c 0x00000000   Number         0  usbd_req.o ABSOLUTE
    ..\\STM32_USB_OTG_Driver\\src\\usb_core.c 0x00000000   Number         0  usb_core.o ABSOLUTE
    ..\\STM32_USB_OTG_Driver\\src\\usb_dcd.c 0x00000000   Number         0  usb_dcd.o ABSOLUTE
    ..\\STM32_USB_OTG_Driver\\src\\usb_dcd_int.c 0x00000000   Number         0  usb_dcd_int.o ABSOLUTE
    dc.s                                     0x00000000   Number         0  dc.o ABSOLUTE
    startup_stm32f40_41xxx.s                 0x00000000   Number         0  startup_stm32f40_41xxx.o ABSOLUTE
    RESET                                    0x08000000   Section      392  startup_stm32f40_41xxx.o(RESET)
    !!!main                                  0x08000188   Section        8  __main.o(!!!main)
    !!!scatter                               0x08000190   Section       52  __scatter.o(!!!scatter)
    !!dczerorl2                              0x080001c4   Section       90  __dczerorl2.o(!!dczerorl2)
    !!handler_zi                             0x08000220   Section       28  __scatter_zi.o(!!handler_zi)
    .ARM.Collect$$libinit$$00000000          0x0800023c   Section        2  libinit.o(.ARM.Collect$$libinit$$00000000)
    .ARM.Collect$$libinit$$00000002          0x0800023e   Section        0  libinit2.o(.ARM.Collect$$libinit$$00000002)
    .ARM.Collect$$libinit$$00000008          0x0800023e   Section        0  libinit2.o(.ARM.Collect$$libinit$$00000008)
    .ARM.Collect$$libinit$$0000000A          0x0800023e   Section        0  libinit2.o(.ARM.Collect$$libinit$$0000000A)
    .ARM.Collect$$libinit$$0000000C          0x0800023e   Section        0  libinit2.o(.ARM.Collect$$libinit$$0000000C)
    .ARM.Collect$$libinit$$0000000F          0x0800023e   Section        0  libinit2.o(.ARM.Collect$$libinit$$0000000F)
    .ARM.Collect$$libinit$$00000011          0x0800023e   Section        0  libinit2.o(.ARM.Collect$$libinit$$00000011)
    .ARM.Collect$$libinit$$00000013          0x0800023e   Section        0  libinit2.o(.ARM.Collect$$libinit$$00000013)
    .ARM.Collect$$libinit$$00000015          0x0800023e   Section        0  libinit2.o(.ARM.Collect$$libinit$$00000015)
    .ARM.Collect$$libinit$$00000017          0x0800023e   Section        0  libinit2.o(.ARM.Collect$$libinit$$00000017)
    .ARM.Collect$$libinit$$00000019          0x0800023e   Section        0  libinit2.o(.ARM.Collect$$libinit$$00000019)
    .ARM.Collect$$libinit$$0000001B          0x0800023e   Section        0  libinit2.o(.ARM.Collect$$libinit$$0000001B)
    .ARM.Collect$$libinit$$0000001D          0x0800023e   Section        0  libinit2.o(.ARM.Collect$$libinit$$0000001D)
    .ARM.Collect$$libinit$$0000001F          0x0800023e   Section        0  libinit2.o(.ARM.Collect$$libinit$$0000001F)
    .ARM.Collect$$libinit$$00000021          0x0800023e   Section        0  libinit2.o(.ARM.Collect$$libinit$$00000021)
    .ARM.Collect$$libinit$$00000023          0x0800023e   Section        0  libinit2.o(.ARM.Collect$$libinit$$00000023)
    .ARM.Collect$$libinit$$0000002A          0x0800023e   Section        0  libinit2.o(.ARM.Collect$$libinit$$0000002A)
    .ARM.Collect$$libinit$$0000002C          0x0800023e   Section        0  libinit2.o(.ARM.Collect$$libinit$$0000002C)
    .ARM.Collect$$libinit$$0000002E          0x0800023e   Section        0  libinit2.o(.ARM.Collect$$libinit$$0000002E)
    .ARM.Collect$$libinit$$00000030          0x0800023e   Section        0  libinit2.o(.ARM.Collect$$libinit$$00000030)
    .ARM.Collect$$libinit$$00000031          0x0800023e   Section        2  libinit2.o(.ARM.Collect$$libinit$$00000031)
    .ARM.Collect$$libshutdown$$00000000      0x08000240   Section        2  libshutdown.o(.ARM.Collect$$libshutdown$$00000000)
    .ARM.Collect$$libshutdown$$00000003      0x08000242   Section        0  libshutdown2.o(.ARM.Collect$$libshutdown$$00000003)
    .ARM.Collect$$libshutdown$$00000006      0x08000242   Section        0  libshutdown2.o(.ARM.Collect$$libshutdown$$00000006)
    .ARM.Collect$$libshutdown$$00000009      0x08000242   Section        0  libshutdown2.o(.ARM.Collect$$libshutdown$$00000009)
    .ARM.Collect$$libshutdown$$0000000B      0x08000242   Section        0  libshutdown2.o(.ARM.Collect$$libshutdown$$0000000B)
    .ARM.Collect$$libshutdown$$0000000E      0x08000242   Section        0  libshutdown2.o(.ARM.Collect$$libshutdown$$0000000E)
    .ARM.Collect$$libshutdown$$0000000F      0x08000242   Section        2  libshutdown2.o(.ARM.Collect$$libshutdown$$0000000F)
    .ARM.Collect$$rtentry$$00000000          0x08000244   Section        0  rtentry.o(.ARM.Collect$$rtentry$$00000000)
    .ARM.Collect$$rtentry$$00000002          0x08000244   Section        0  rtentry2.o(.ARM.Collect$$rtentry$$00000002)
    .ARM.Collect$$rtentry$$00000004          0x08000244   Section        6  rtentry4.o(.ARM.Collect$$rtentry$$00000004)
    .ARM.Collect$$rtentry$$00000009          0x0800024a   Section        0  rtentry2.o(.ARM.Collect$$rtentry$$00000009)
    .ARM.Collect$$rtentry$$0000000A          0x0800024a   Section        4  rtentry2.o(.ARM.Collect$$rtentry$$0000000A)
    .ARM.Collect$$rtentry$$0000000C          0x0800024e   Section        0  rtentry2.o(.ARM.Collect$$rtentry$$0000000C)
    .ARM.Collect$$rtentry$$0000000D          0x0800024e   Section        8  rtentry2.o(.ARM.Collect$$rtentry$$0000000D)
    .ARM.Collect$$rtexit$$00000000           0x08000256   Section        2  rtexit.o(.ARM.Collect$$rtexit$$00000000)
    .ARM.Collect$$rtexit$$00000002           0x08000258   Section        0  rtexit2.o(.ARM.Collect$$rtexit$$00000002)
    .ARM.Collect$$rtexit$$00000003           0x08000258   Section        4  rtexit2.o(.ARM.Collect$$rtexit$$00000003)
    .ARM.Collect$$rtexit$$00000004           0x0800025c   Section        6  rtexit2.o(.ARM.Collect$$rtexit$$00000004)
    .text                                    0x08000264   Section       64  startup_stm32f40_41xxx.o(.text)
    .text                                    0x080002a4   Section        0  system_stm32f4xx.o(.text)
    SetSysClock                              0x080002a5   Thumb Code   266  system_stm32f4xx.o(.text)
    .text                                    0x080004d8   Section        0  misc.o(.text)
    .text                                    0x080005bc   Section        0  stm32f4xx_dac.o(.text)
    .text                                    0x080007cc   Section        0  stm32f4xx_dma.o(.text)
    .text                                    0x08000b70   Section        0  stm32f4xx_exti.o(.text)
    .text                                    0x08000c8c   Section        0  stm32f4xx_gpio.o(.text)
    .text                                    0x08000ee8   Section        0  stm32f4xx_i2c.o(.text)
    .text                                    0x08001310   Section        0  stm32f4xx_rcc.o(.text)
    .text                                    0x08001898   Section        0  stm32f4xx_spi.o(.text)
    .text                                    0x08001c8c   Section        0  stm32f4xx_syscfg.o(.text)
    .text                                    0x08001d18   Section        0  usbd_audio_core.o(.text)
    usbd_audio_Init                          0x08001d19   Thumb Code    54  usbd_audio_core.o(.text)
    usbd_audio_DeInit                        0x08001d4f   Thumb Code    32  usbd_audio_core.o(.text)
    AUDIO_Req_SetCurrent                     0x08001d6f   Thumb Code    42  usbd_audio_core.o(.text)
    AUDIO_Req_GetCurrent                     0x08001d99   Thumb Code    18  usbd_audio_core.o(.text)
    usbd_audio_Setup                         0x08001dab   Thumb Code   168  usbd_audio_core.o(.text)
    usbd_audio_EP0_RxReady                   0x08001e53   Thumb Code    44  usbd_audio_core.o(.text)
    usbd_audio_DataIn                        0x08001e7f   Thumb Code     6  usbd_audio_core.o(.text)
    usbd_audio_DataOut                       0x08001e85   Thumb Code   114  usbd_audio_core.o(.text)
    usbd_audio_SOF                           0x08001ef7   Thumb Code    96  usbd_audio_core.o(.text)
    usbd_audio_OUT_Incplt                    0x08001f57   Thumb Code     6  usbd_audio_core.o(.text)
    USBD_audio_GetCfgDesc                    0x08001f5d   Thumb Code    12  usbd_audio_core.o(.text)
    .text                                    0x08001f9c   Section        0  usbd_audio_out_if.o(.text)
    Init                                     0x08001f9d   Thumb Code    52  usbd_audio_out_if.o(.text)
    DeInit                                   0x08001fd1   Thumb Code    10  usbd_audio_out_if.o(.text)
    AudioCmd                                 0x08001fdb   Thumb Code   212  usbd_audio_out_if.o(.text)
    VolumeCtl                                0x080020af   Thumb Code     6  usbd_audio_out_if.o(.text)
    MuteCtl                                  0x080020b5   Thumb Code    26  usbd_audio_out_if.o(.text)
    PeriodicTC                               0x080020cf   Thumb Code     6  usbd_audio_out_if.o(.text)
    GetState                                 0x080020d5   Thumb Code     6  usbd_audio_out_if.o(.text)
    .text                                    0x080020e4   Section        0  usbd_core.o(.text)
    USBD_SetupStage                          0x0800212d   Thumb Code    84  usbd_core.o(.text)
    USBD_DataOutStage                        0x08002181   Thumb Code   150  usbd_core.o(.text)
    USBD_DataInStage                         0x08002217   Thumb Code   184  usbd_core.o(.text)
    USBD_Reset                               0x080022cf   Thumb Code    50  usbd_core.o(.text)
    USBD_Resume                              0x08002301   Thumb Code    24  usbd_core.o(.text)
    USBD_Suspend                             0x08002319   Thumb Code    24  usbd_core.o(.text)
    USBD_SOF                                 0x08002331   Thumb Code    26  usbd_core.o(.text)
    USBD_IsoINIncomplete                     0x0800237f   Thumb Code    18  usbd_core.o(.text)
    USBD_IsoOUTIncomplete                    0x08002391   Thumb Code    18  usbd_core.o(.text)
    .text                                    0x080023a2   Section        0  usbd_ioreq.o(.text)
    .text                                    0x08002498   Section        0  usbd_req.o(.text)
    USBD_ClrFeature                          0x080024d1   Thumb Code    72  usbd_req.o(.text)
    USBD_SetFeature                          0x08002519   Thumb Code   152  usbd_req.o(.text)
    USBD_GetStatus                           0x080025b1   Thumb Code    72  usbd_req.o(.text)
    USBD_GetConfig                           0x080025f9   Thumb Code    78  usbd_req.o(.text)
    USBD_SetConfig                           0x08002647   Thumb Code   204  usbd_req.o(.text)
    USBD_SetAddress                          0x08002713   Thumb Code    92  usbd_req.o(.text)
    USBD_GetDescriptor                       0x0800276f   Thumb Code   290  usbd_req.o(.text)
    USBD_GetLen                              0x08002afd   Thumb Code    20  usbd_req.o(.text)
    .text                                    0x08002b68   Section        0  usb_core.o(.text)
    USB_OTG_EnableCommonInt                  0x08002b69   Thumb Code    48  usb_core.o(.text)
    USB_OTG_CoreReset                        0x08002b99   Thumb Code   104  usb_core.o(.text)
    .text                                    0x08003be6   Section        0  usb_dcd.o(.text)
    .text                                    0x08003f64   Section        0  usb_dcd_int.o(.text)
    DCD_IsoOUTIncomplete_ISR                 0x08003f65   Thumb Code    40  usb_dcd_int.o(.text)
    DCD_IsoINIncomplete_ISR                  0x08003f8d   Thumb Code    40  usb_dcd_int.o(.text)
    DCD_HandleEnumDone_ISR                   0x08003fb5   Thumb Code   102  usb_dcd_int.o(.text)
    DCD_HandleUsbReset_ISR                   0x0800401b   Thumb Code   284  usb_dcd_int.o(.text)
    DCD_HandleRxStatusQueueLevel_ISR         0x08004137   Thumb Code   176  usb_dcd_int.o(.text)
    DCD_HandleSof_ISR                        0x080041e7   Thumb Code    38  usb_dcd_int.o(.text)
    DCD_HandleUSBSuspend_ISR                 0x0800420d   Thumb Code   126  usb_dcd_int.o(.text)
    DCD_HandleResume_ISR                     0x0800428b   Thumb Code   100  usb_dcd_int.o(.text)
    DCD_WriteEmptyTxFifo                     0x080042ef   Thumb Code   154  usb_dcd_int.o(.text)
    DCD_ReadDevInEP                          0x08004389   Thumb Code    40  usb_dcd_int.o(.text)
    DCD_HandleInEP_ISR                       0x080043b1   Thumb Code   386  usb_dcd_int.o(.text)
    DCD_HandleOutEP_ISR                      0x08004533   Thumb Code   286  usb_dcd_int.o(.text)
    .text                                    0x08004734   Section        0  main.o(.text)
    .text                                    0x08004788   Section        0  stm32f4xx_it.o(.text)
    .text                                    0x080047dc   Section        0  usb_bsp.o(.text)
    .text                                    0x080048dc   Section        0  usbd_desc.o(.text)
    .text                                    0x08004a34   Section        0  usbd_usr.o(.text)
    .text                                    0x08004ab8   Section        0  stm32f4_discovery.o(.text)
    .text                                    0x08004bfc   Section        0  stm32f4_discovery_audio_codec.o(.text)
    Audio_MAL_Init                           0x08004c99   Thumb Code    54  stm32f4_discovery_audio_codec.o(.text)
    Codec_AudioInterface_Init                0x08004ccf   Thumb Code   102  stm32f4_discovery_audio_codec.o(.text)
    Codec_ReadRegister                       0x08004d39   Thumb Code   410  stm32f4_discovery_audio_codec.o(.text)
    Codec_WriteRegister                      0x08004ed3   Thumb Code   354  stm32f4_discovery_audio_codec.o(.text)
    Codec_VolumeCtrl                         0x08005035   Thumb Code    72  stm32f4_discovery_audio_codec.o(.text)
    Codec_CtrlInterface_Init                 0x0800507d   Thumb Code    72  stm32f4_discovery_audio_codec.o(.text)
    Delay                                    0x080050c5   Thumb Code    18  stm32f4_discovery_audio_codec.o(.text)
    Codec_Reset                              0x080050d7   Thumb Code    32  stm32f4_discovery_audio_codec.o(.text)
    Codec_GPIO_Init                          0x080050f7   Thumb Code   268  stm32f4_discovery_audio_codec.o(.text)
    Codec_Init                               0x08005203   Thumb Code   224  stm32f4_discovery_audio_codec.o(.text)
    Codec_AudioInterface_DeInit              0x0800531d   Thumb Code    28  stm32f4_discovery_audio_codec.o(.text)
    Codec_CtrlInterface_DeInit               0x08005339   Thumb Code     2  stm32f4_discovery_audio_codec.o(.text)
    Codec_GPIO_DeInit                        0x0800533b   Thumb Code   100  stm32f4_discovery_audio_codec.o(.text)
    Codec_DeInit                             0x0800539f   Thumb Code    34  stm32f4_discovery_audio_codec.o(.text)
    Audio_MAL_DeInit                         0x080053c1   Thumb Code    22  stm32f4_discovery_audio_codec.o(.text)
    Codec_Play                               0x080054d7   Thumb Code     4  stm32f4_discovery_audio_codec.o(.text)
    Audio_MAL_PauseResume                    0x08005549   Thumb Code    76  stm32f4_discovery_audio_codec.o(.text)
    Codec_Mute                               0x08005595   Thumb Code    38  stm32f4_discovery_audio_codec.o(.text)
    Codec_PauseResume                        0x080055bb   Thumb Code    62  stm32f4_discovery_audio_codec.o(.text)
    Audio_MAL_Stop                           0x08005615   Thumb Code    56  stm32f4_discovery_audio_codec.o(.text)
    Codec_Stop                               0x0800564d   Thumb Code    60  stm32f4_discovery_audio_codec.o(.text)
    Audio_MAL_IRQHandler                     0x080056d5   Thumb Code    10  stm32f4_discovery_audio_codec.o(.text)
    .text                                    0x08005830   Section        0  heapauxi.o(.text)
    .text                                    0x08005836   Section       74  sys_stackheap_outer.o(.text)
    .text                                    0x08005880   Section        0  exit.o(.text)
    .text                                    0x0800588c   Section        8  libspace.o(.text)
    .text                                    0x08005894   Section        0  sys_exit.o(.text)
    .text                                    0x080058a0   Section        2  use_no_semi.o(.text)
    .text                                    0x080058a2   Section        0  indicate_semi.o(.text)
    .constdata                               0x080058a4   Section       37  stm32f4_discovery.o(.constdata)
    .data                                    0x20000000   Section       20  system_stm32f4xx.o(.data)
    .data                                    0x20000014   Section       16  stm32f4xx_rcc.o(.data)
    APBAHBPrescTable                         0x20000014   Data          16  stm32f4xx_rcc.o(.data)
    .data                                    0x20000024   Section      181  usbd_audio_core.o(.data)
    PlayFlag                                 0x20000038   Data           4  usbd_audio_core.o(.data)
    usbd_audio_AltSet                        0x2000003c   Data           4  usbd_audio_core.o(.data)
    usbd_audio_CfgDesc                       0x2000006c   Data         109  usbd_audio_core.o(.data)
    .data                                    0x200000dc   Section       36  usbd_audio_out_if.o(.data)
    AudioState                               0x200000f8   Data           1  usbd_audio_out_if.o(.data)
    Initialized                              0x200000fc   Data           4  usbd_audio_out_if.o(.data)
    .data                                    0x20000100   Section       48  usbd_core.o(.data)
    .data                                    0x20000130   Section       13  usbd_req.o(.data)
    cfgidx                                   0x2000013c   Data           1  usbd_req.o(.data)
    .data                                    0x20000140   Section       14  main.o(.data)
    .data                                    0x20000150   Section       60  usbd_desc.o(.data)
    .data                                    0x2000018c   Section       28  usbd_usr.o(.data)
    .data                                    0x200001a8   Section       24  stm32f4_discovery.o(.data)
    .data                                    0x200001c0   Section       76  stm32f4_discovery_audio_codec.o(.data)
    tmp                                      0x200001fc   Data           1  stm32f4_discovery_audio_codec.o(.data)
    udata                                    0x200001fe   Data           2  stm32f4_discovery_audio_codec.o(.data)
    .bss                                     0x2000020c   Section     1600  usbd_audio_core.o(.bss)
    .bss                                     0x2000084c   Section      200  usbd_req.o(.bss)
    .bss                                     0x20000914   Section     1520  main.o(.bss)
    .bss                                     0x20000f04   Section      120  stm32f4_discovery_audio_codec.o(.bss)
    .bss                                     0x20000f7c   Section       96  libspace.o(.bss)
    HEAP                                     0x20000fe0   Section      512  startup_stm32f40_41xxx.o(HEAP)
    Heap_Mem                                 0x20000fe0   Data         512  startup_stm32f40_41xxx.o(HEAP)
    STACK                                    0x200011e0   Section     1024  startup_stm32f40_41xxx.o(STACK)
    Stack_Mem                                0x200011e0   Data        1024  startup_stm32f40_41xxx.o(STACK)
    __initial_sp                             0x200015e0   Data           0  startup_stm32f40_41xxx.o(STACK)

    Global Symbols

    Symbol Name                              Value     Ov Type        Size  Object(Section)

    BuildAttributes$$THM_ISAv4$E$P$D$K$B$S$7EM$PE$A:L22UL41UL21$X:L11$S22US41US21$IEEE1$IW$USESV6$~STKCKD$USESV7$~SHL$OSPACE$ROPI$EBA8$UX$STANDARDLIB$REQ8$PRES8$EABIv2 0x00000000   Number         0  anon$$obj.o ABSOLUTE
    __ARM_use_no_argv                        0x00000000   Number         0  main.o ABSOLUTE
    __ARM_exceptions_init                     - Undefined Weak Reference
    __alloca_initialize                       - Undefined Weak Reference
    __cpp_initialize__aeabi_                  - Undefined Weak Reference
    __cxa_finalize                            - Undefined Weak Reference
    __rt_locale                               - Undefined Weak Reference
    __sigvec_lookup                           - Undefined Weak Reference
    _atexit_init                              - Undefined Weak Reference
    _call_atexit_fns                          - Undefined Weak Reference
    _clock_init                               - Undefined Weak Reference
    _fp_trap_init                             - Undefined Weak Reference
    _fp_trap_shutdown                         - Undefined Weak Reference
    _get_lc_collate                           - Undefined Weak Reference
    _get_lc_ctype                             - Undefined Weak Reference
    _get_lc_monetary                          - Undefined Weak Reference
    _get_lc_numeric                           - Undefined Weak Reference
    _get_lc_time                              - Undefined Weak Reference
    _getenv_init                              - Undefined Weak Reference
    _handle_redirection                       - Undefined Weak Reference
    _init_alloc                               - Undefined Weak Reference
    _init_user_alloc                          - Undefined Weak Reference
    _initio                                   - Undefined Weak Reference
    _rand_init                                - Undefined Weak Reference
    _signal_finish                            - Undefined Weak Reference
    _signal_init                              - Undefined Weak Reference
    _terminate_alloc                          - Undefined Weak Reference
    _terminate_user_alloc                     - Undefined Weak Reference
    _terminateio                              - Undefined Weak Reference
    __Vectors_Size                           0x00000188   Number         0  startup_stm32f40_41xxx.o ABSOLUTE
    __Vectors                                0x08000000   Data           4  startup_stm32f40_41xxx.o(RESET)
    __Vectors_End                            0x08000188   Data           0  startup_stm32f40_41xxx.o(RESET)
    __main                                   0x08000189   Thumb Code     8  __main.o(!!!main)
    __scatterload                            0x08000191   Thumb Code     0  __scatter.o(!!!scatter)
    __scatterload_rt2                        0x08000191   Thumb Code    44  __scatter.o(!!!scatter)
    __scatterload_rt2_thumb_only             0x08000191   Thumb Code     0  __scatter.o(!!!scatter)
    __scatterload_null                       0x0800019f   Thumb Code     0  __scatter.o(!!!scatter)
    __decompress                             0x080001c5   Thumb Code    90  __dczerorl2.o(!!dczerorl2)
    __decompress1                            0x080001c5   Thumb Code     0  __dczerorl2.o(!!dczerorl2)
    __scatterload_zeroinit                   0x08000221   Thumb Code    28  __scatter_zi.o(!!handler_zi)
    __rt_lib_init                            0x0800023d   Thumb Code     0  libinit.o(.ARM.Collect$$libinit$$00000000)
    __rt_lib_init_alloca_1                   0x0800023f   Thumb Code     0  libinit2.o(.ARM.Collect$$libinit$$0000002C)
    __rt_lib_init_argv_1                     0x0800023f   Thumb Code     0  libinit2.o(.ARM.Collect$$libinit$$0000002A)
    __rt_lib_init_atexit_1                   0x0800023f   Thumb Code     0  libinit2.o(.ARM.Collect$$libinit$$00000019)
    __rt_lib_init_clock_1                    0x0800023f   Thumb Code     0  libinit2.o(.ARM.Collect$$libinit$$0000001F)
    __rt_lib_init_cpp_1                      0x0800023f   Thumb Code     0  libinit2.o(.ARM.Collect$$libinit$$00000030)
    __rt_lib_init_exceptions_1               0x0800023f   Thumb Code     0  libinit2.o(.ARM.Collect$$libinit$$0000002E)
    __rt_lib_init_fp_1                       0x0800023f   Thumb Code     0  libinit2.o(.ARM.Collect$$libinit$$00000002)
    __rt_lib_init_fp_trap_1                  0x0800023f   Thumb Code     0  libinit2.o(.ARM.Collect$$libinit$$0000001D)
    __rt_lib_init_getenv_1                   0x0800023f   Thumb Code     0  libinit2.o(.ARM.Collect$$libinit$$00000021)
    __rt_lib_init_heap_1                     0x0800023f   Thumb Code     0  libinit2.o(.ARM.Collect$$libinit$$00000008)
    __rt_lib_init_lc_collate_1               0x0800023f   Thumb Code     0  libinit2.o(.ARM.Collect$$libinit$$0000000F)
    __rt_lib_init_lc_ctype_1                 0x0800023f   Thumb Code     0  libinit2.o(.ARM.Collect$$libinit$$00000011)
    __rt_lib_init_lc_monetary_1              0x0800023f   Thumb Code     0  libinit2.o(.ARM.Collect$$libinit$$00000013)
    __rt_lib_init_lc_numeric_1               0x0800023f   Thumb Code     0  libinit2.o(.ARM.Collect$$libinit$$00000015)
    __rt_lib_init_lc_time_1                  0x0800023f   Thumb Code     0  libinit2.o(.ARM.Collect$$libinit$$00000017)
    __rt_lib_init_rand_1                     0x0800023f   Thumb Code     0  libinit2.o(.ARM.Collect$$libinit$$0000000C)
    __rt_lib_init_return                     0x0800023f   Thumb Code     0  libinit2.o(.ARM.Collect$$libinit$$00000031)
    __rt_lib_init_signal_1                   0x0800023f   Thumb Code     0  libinit2.o(.ARM.Collect$$libinit$$0000001B)
    __rt_lib_init_stdio_1                    0x0800023f   Thumb Code     0  libinit2.o(.ARM.Collect$$libinit$$00000023)
    __rt_lib_init_user_alloc_1               0x0800023f   Thumb Code     0  libinit2.o(.ARM.Collect$$libinit$$0000000A)
    __rt_lib_shutdown                        0x08000241   Thumb Code     0  libshutdown.o(.ARM.Collect$$libshutdown$$00000000)
    __rt_lib_shutdown_fp_trap_1              0x08000243   Thumb Code     0  libshutdown2.o(.ARM.Collect$$libshutdown$$00000006)
    __rt_lib_shutdown_heap_1                 0x08000243   Thumb Code     0  libshutdown2.o(.ARM.Collect$$libshutdown$$0000000E)
    __rt_lib_shutdown_return                 0x08000243   Thumb Code     0  libshutdown2.o(.ARM.Collect$$libshutdown$$0000000F)
    __rt_lib_shutdown_signal_1               0x08000243   Thumb Code     0  libshutdown2.o(.ARM.Collect$$libshutdown$$00000009)
    __rt_lib_shutdown_stdio_1                0x08000243   Thumb Code     0  libshutdown2.o(.ARM.Collect$$libshutdown$$00000003)
    __rt_lib_shutdown_user_alloc_1           0x08000243   Thumb Code     0  libshutdown2.o(.ARM.Collect$$libshutdown$$0000000B)
    __rt_entry                               0x08000245   Thumb Code     0  rtentry.o(.ARM.Collect$$rtentry$$00000000)
    __rt_entry_presh_1                       0x08000245   Thumb Code     0  rtentry2.o(.ARM.Collect$$rtentry$$00000002)
    __rt_entry_sh                            0x08000245   Thumb Code     0  rtentry4.o(.ARM.Collect$$rtentry$$00000004)
    __rt_entry_li                            0x0800024b   Thumb Code     0  rtentry2.o(.ARM.Collect$$rtentry$$0000000A)
    __rt_entry_postsh_1                      0x0800024b   Thumb Code     0  rtentry2.o(.ARM.Collect$$rtentry$$00000009)
    __rt_entry_main                          0x0800024f   Thumb Code     0  rtentry2.o(.ARM.Collect$$rtentry$$0000000D)
    __rt_entry_postli_1                      0x0800024f   Thumb Code     0  rtentry2.o(.ARM.Collect$$rtentry$$0000000C)
    __rt_exit                                0x08000257   Thumb Code     0  rtexit.o(.ARM.Collect$$rtexit$$00000000)
    __rt_exit_ls                             0x08000259   Thumb Code     0  rtexit2.o(.ARM.Collect$$rtexit$$00000003)
    __rt_exit_prels_1                        0x08000259   Thumb Code     0  rtexit2.o(.ARM.Collect$$rtexit$$00000002)
    __rt_exit_exit                           0x0800025d   Thumb Code     0  rtexit2.o(.ARM.Collect$$rtexit$$00000004)
    Reset_Handler                            0x08000265   Thumb Code     8  startup_stm32f40_41xxx.o(.text)
    ADC_IRQHandler                           0x0800027f   Thumb Code     0  startup_stm32f40_41xxx.o(.text)
    CAN1_RX0_IRQHandler                      0x0800027f   Thumb Code     0  startup_stm32f40_41xxx.o(.text)
    CAN1_RX1_IRQHandler                      0x0800027f   Thumb Code     0  startup_stm32f40_41xxx.o(.text)
    CAN1_SCE_IRQHandler                      0x0800027f   Thumb Code     0  startup_stm32f40_41xxx.o(.text)
    CAN1_TX_IRQHandler                       0x0800027f   Thumb Code     0  startup_stm32f40_41xxx.o(.text)
    CAN2_RX0_IRQHandler                      0x0800027f   Thumb Code     0  startup_stm32f40_41xxx.o(.text)
    CAN2_RX1_IRQHandler                      0x0800027f   Thumb Code     0  startup_stm32f40_41xxx.o(.text)
    CAN2_SCE_IRQHandler                      0x0800027f   Thumb Code     0  startup_stm32f40_41xxx.o(.text)
    CAN2_TX_IRQHandler                       0x0800027f   Thumb Code     0  startup_stm32f40_41xxx.o(.text)
    CRYP_IRQHandler                          0x0800027f   Thumb Code     0  startup_stm32f40_41xxx.o(.text)
    DCMI_IRQHandler                          0x0800027f   Thumb Code     0  startup_stm32f40_41xxx.o(.text)
    DMA1_Stream1_IRQHandler                  0x0800027f   Thumb Code     0  startup_stm32f40_41xxx.o(.text)
    DMA1_Stream2_IRQHandler                  0x0800027f   Thumb Code     0  startup_stm32f40_41xxx.o(.text)
    DMA1_Stream3_IRQHandler                  0x0800027f   Thumb Code     0  startup_stm32f40_41xxx.o(.text)
    DMA1_Stream4_IRQHandler                  0x0800027f   Thumb Code     0  startup_stm32f40_41xxx.o(.text)
    DMA1_Stream5_IRQHandler                  0x0800027f   Thumb Code     0  startup_stm32f40_41xxx.o(.text)
    DMA1_Stream6_IRQHandler                  0x0800027f   Thumb Code     0  startup_stm32f40_41xxx.o(.text)
    DMA2_Stream0_IRQHandler                  0x0800027f   Thumb Code     0  startup_stm32f40_41xxx.o(.text)
    DMA2_Stream1_IRQHandler                  0x0800027f   Thumb Code     0  startup_stm32f40_41xxx.o(.text)
    DMA2_Stream2_IRQHandler                  0x0800027f   Thumb Code     0  startup_stm32f40_41xxx.o(.text)
    DMA2_Stream3_IRQHandler                  0x0800027f   Thumb Code     0  startup_stm32f40_41xxx.o(.text)
    DMA2_Stream4_IRQHandler                  0x0800027f   Thumb Code     0  startup_stm32f40_41xxx.o(.text)
    DMA2_Stream5_IRQHandler                  0x0800027f   Thumb Code     0  startup_stm32f40_41xxx.o(.text)
    DMA2_Stream6_IRQHandler                  0x0800027f   Thumb Code     0  startup_stm32f40_41xxx.o(.text)
    DMA2_Stream7_IRQHandler                  0x0800027f   Thumb Code     0  startup_stm32f40_41xxx.o(.text)
    ETH_IRQHandler                           0x0800027f   Thumb Code     0  startup_stm32f40_41xxx.o(.text)
    ETH_WKUP_IRQHandler                      0x0800027f   Thumb Code     0  startup_stm32f40_41xxx.o(.text)
    EXTI0_IRQHandler                         0x0800027f   Thumb Code     0  startup_stm32f40_41xxx.o(.text)
    EXTI15_10_IRQHandler                     0x0800027f   Thumb Code     0  startup_stm32f40_41xxx.o(.text)
    EXTI1_IRQHandler                         0x0800027f   Thumb Code     0  startup_stm32f40_41xxx.o(.text)
    EXTI2_IRQHandler                         0x0800027f   Thumb Code     0  startup_stm32f40_41xxx.o(.text)
    EXTI3_IRQHandler                         0x0800027f   Thumb Code     0  startup_stm32f40_41xxx.o(.text)
    EXTI4_IRQHandler                         0x0800027f   Thumb Code     0  startup_stm32f40_41xxx.o(.text)
    EXTI9_5_IRQHandler                       0x0800027f   Thumb Code     0  startup_stm32f40_41xxx.o(.text)
    FLASH_IRQHandler                         0x0800027f   Thumb Code     0  startup_stm32f40_41xxx.o(.text)
    FPU_IRQHandler                           0x0800027f   Thumb Code     0  startup_stm32f40_41xxx.o(.text)
    FSMC_IRQHandler                          0x0800027f   Thumb Code     0  startup_stm32f40_41xxx.o(.text)
    HASH_RNG_IRQHandler                      0x0800027f   Thumb Code     0  startup_stm32f40_41xxx.o(.text)
    I2C1_ER_IRQHandler                       0x0800027f   Thumb Code     0  startup_stm32f40_41xxx.o(.text)
    I2C1_EV_IRQHandler                       0x0800027f   Thumb Code     0  startup_stm32f40_41xxx.o(.text)
    I2C2_ER_IRQHandler                       0x0800027f   Thumb Code     0  startup_stm32f40_41xxx.o(.text)
    I2C2_EV_IRQHandler                       0x0800027f   Thumb Code     0  startup_stm32f40_41xxx.o(.text)
    I2C3_ER_IRQHandler                       0x0800027f   Thumb Code     0  startup_stm32f40_41xxx.o(.text)
    I2C3_EV_IRQHandler                       0x0800027f   Thumb Code     0  startup_stm32f40_41xxx.o(.text)
    OTG_HS_EP1_IN_IRQHandler                 0x0800027f   Thumb Code     0  startup_stm32f40_41xxx.o(.text)
    OTG_HS_EP1_OUT_IRQHandler                0x0800027f   Thumb Code     0  startup_stm32f40_41xxx.o(.text)
    OTG_HS_IRQHandler                        0x0800027f   Thumb Code     0  startup_stm32f40_41xxx.o(.text)
    OTG_HS_WKUP_IRQHandler                   0x0800027f   Thumb Code     0  startup_stm32f40_41xxx.o(.text)
    PVD_IRQHandler                           0x0800027f   Thumb Code     0  startup_stm32f40_41xxx.o(.text)
    RCC_IRQHandler                           0x0800027f   Thumb Code     0  startup_stm32f40_41xxx.o(.text)
    RTC_Alarm_IRQHandler                     0x0800027f   Thumb Code     0  startup_stm32f40_41xxx.o(.text)
    RTC_WKUP_IRQHandler                      0x0800027f   Thumb Code     0  startup_stm32f40_41xxx.o(.text)
    SDIO_IRQHandler                          0x0800027f   Thumb Code     0  startup_stm32f40_41xxx.o(.text)
    SPI1_IRQHandler                          0x0800027f   Thumb Code     0  startup_stm32f40_41xxx.o(.text)
    SPI2_IRQHandler                          0x0800027f   Thumb Code     0  startup_stm32f40_41xxx.o(.text)
    TAMP_STAMP_IRQHandler                    0x0800027f   Thumb Code     0  startup_stm32f40_41xxx.o(.text)
    TIM1_BRK_TIM9_IRQHandler                 0x0800027f   Thumb Code     0  startup_stm32f40_41xxx.o(.text)
    TIM1_CC_IRQHandler                       0x0800027f   Thumb Code     0  startup_stm32f40_41xxx.o(.text)
    TIM1_TRG_COM_TIM11_IRQHandler            0x0800027f   Thumb Code     0  startup_stm32f40_41xxx.o(.text)
    TIM1_UP_TIM10_IRQHandler                 0x0800027f   Thumb Code     0  startup_stm32f40_41xxx.o(.text)
    TIM2_IRQHandler                          0x0800027f   Thumb Code     0  startup_stm32f40_41xxx.o(.text)
    TIM3_IRQHandler                          0x0800027f   Thumb Code     0  startup_stm32f40_41xxx.o(.text)
    TIM4_IRQHandler                          0x0800027f   Thumb Code     0  startup_stm32f40_41xxx.o(.text)
    TIM5_IRQHandler                          0x0800027f   Thumb Code     0  startup_stm32f40_41xxx.o(.text)
    TIM6_DAC_IRQHandler                      0x0800027f   Thumb Code     0  startup_stm32f40_41xxx.o(.text)
    TIM7_IRQHandler                          0x0800027f   Thumb Code     0  startup_stm32f40_41xxx.o(.text)
    TIM8_BRK_TIM12_IRQHandler                0x0800027f   Thumb Code     0  startup_stm32f40_41xxx.o(.text)
    TIM8_CC_IRQHandler                       0x0800027f   Thumb Code     0  startup_stm32f40_41xxx.o(.text)
    TIM8_TRG_COM_TIM14_IRQHandler            0x0800027f   Thumb Code     0  startup_stm32f40_41xxx.o(.text)
    TIM8_UP_TIM13_IRQHandler                 0x0800027f   Thumb Code     0  startup_stm32f40_41xxx.o(.text)
    UART4_IRQHandler                         0x0800027f   Thumb Code     0  startup_stm32f40_41xxx.o(.text)
    UART5_IRQHandler                         0x0800027f   Thumb Code     0  startup_stm32f40_41xxx.o(.text)
    USART1_IRQHandler                        0x0800027f   Thumb Code     0  startup_stm32f40_41xxx.o(.text)
    USART2_IRQHandler                        0x0800027f   Thumb Code     0  startup_stm32f40_41xxx.o(.text)
    USART3_IRQHandler                        0x0800027f   Thumb Code     0  startup_stm32f40_41xxx.o(.text)
    USART6_IRQHandler                        0x0800027f   Thumb Code     0  startup_stm32f40_41xxx.o(.text)
    WWDG_IRQHandler                          0x0800027f   Thumb Code     0  startup_stm32f40_41xxx.o(.text)
    __user_initial_stackheap                 0x08000281   Thumb Code     0  startup_stm32f40_41xxx.o(.text)
    SystemInit                               0x080003af   Thumb Code    74  system_stm32f4xx.o(.text)
    SystemCoreClockUpdate                    0x080003f9   Thumb Code   174  system_stm32f4xx.o(.text)
    NVIC_PriorityGroupConfig                 0x080004d9   Thumb Code    10  misc.o(.text)
    NVIC_Init                                0x080004e3   Thumb Code   108  misc.o(.text)
    NVIC_SetVectorTable                      0x0800054f   Thumb Code    14  misc.o(.text)
    NVIC_SystemLPConfig                      0x0800055d   Thumb Code    34  misc.o(.text)
    SysTick_CLKSourceConfig                  0x0800057f   Thumb Code    40  misc.o(.text)
    DAC_DeInit                               0x080005bd   Thumb Code    22  stm32f4xx_dac.o(.text)
    DAC_Init                                 0x080005d3   Thumb Code    46  stm32f4xx_dac.o(.text)
    DAC_StructInit                           0x08000601   Thumb Code    12  stm32f4xx_dac.o(.text)
    DAC_Cmd                                  0x0800060d   Thumb Code    34  stm32f4xx_dac.o(.text)
    DAC_SoftwareTriggerCmd                   0x0800062f   Thumb Code    48  stm32f4xx_dac.o(.text)
    DAC_DualSoftwareTriggerCmd               0x0800065f   Thumb Code    38  stm32f4xx_dac.o(.text)
    DAC_WaveGenerationCmd                    0x08000685   Thumb Code    36  stm32f4xx_dac.o(.text)
    DAC_SetChannel1Data                      0x080006a9   Thumb Code    26  stm32f4xx_dac.o(.text)
    DAC_SetChannel2Data                      0x080006c3   Thumb Code    26  stm32f4xx_dac.o(.text)
    DAC_SetDualChannelData                   0x080006dd   Thumb Code    32  stm32f4xx_dac.o(.text)
    DAC_GetDataOutputValue                   0x080006fd   Thumb Code    32  stm32f4xx_dac.o(.text)
    DAC_DMACmd                               0x0800071d   Thumb Code    38  stm32f4xx_dac.o(.text)
    DAC_ITConfig                             0x08000743   Thumb Code    36  stm32f4xx_dac.o(.text)
    DAC_GetFlagStatus                        0x08000767   Thumb Code    28  stm32f4xx_dac.o(.text)
    DAC_ClearFlag                            0x08000783   Thumb Code    12  stm32f4xx_dac.o(.text)
    DAC_GetITStatus                          0x0800078f   Thumb Code    44  stm32f4xx_dac.o(.text)
    DAC_ClearITPendingBit                    0x080007bb   Thumb Code    12  stm32f4xx_dac.o(.text)
    DMA_DeInit                               0x080007cd   Thumb Code   324  stm32f4xx_dma.o(.text)
    DMA_Init                                 0x08000911   Thumb Code    82  stm32f4xx_dma.o(.text)
    DMA_StructInit                           0x08000963   Thumb Code    34  stm32f4xx_dma.o(.text)
    DMA_Cmd                                  0x08000985   Thumb Code    22  stm32f4xx_dma.o(.text)
    DMA_PeriphIncOffsetSizeConfig            0x0800099b   Thumb Code    22  stm32f4xx_dma.o(.text)
    DMA_FlowControllerConfig                 0x080009b1   Thumb Code    22  stm32f4xx_dma.o(.text)
    DMA_SetCurrDataCounter                   0x080009c7   Thumb Code     4  stm32f4xx_dma.o(.text)
    DMA_GetCurrDataCounter                   0x080009cb   Thumb Code     8  stm32f4xx_dma.o(.text)
    DMA_DoubleBufferModeConfig               0x080009d3   Thumb Code    24  stm32f4xx_dma.o(.text)
    DMA_DoubleBufferModeCmd                  0x080009eb   Thumb Code    22  stm32f4xx_dma.o(.text)
    DMA_MemoryTargetConfig                   0x08000a01   Thumb Code    10  stm32f4xx_dma.o(.text)
    DMA_GetCurrentMemoryTarget               0x08000a0b   Thumb Code    20  stm32f4xx_dma.o(.text)
    DMA_GetCmdStatus                         0x08000a1f   Thumb Code    20  stm32f4xx_dma.o(.text)
    DMA_GetFIFOStatus                        0x08000a33   Thumb Code    12  stm32f4xx_dma.o(.text)
    DMA_GetFlagStatus                        0x08000a3f   Thumb Code    54  stm32f4xx_dma.o(.text)
    DMA_ClearFlag                            0x08000a75   Thumb Code    40  stm32f4xx_dma.o(.text)
    DMA_ITConfig                             0x08000a9d   Thumb Code    58  stm32f4xx_dma.o(.text)
    DMA_GetITStatus                          0x08000ad7   Thumb Code    82  stm32f4xx_dma.o(.text)
    DMA_ClearITPendingBit                    0x08000b29   Thumb Code    40  stm32f4xx_dma.o(.text)
    EXTI_DeInit                              0x08000b71   Thumb Code    28  stm32f4xx_exti.o(.text)
    EXTI_Init                                0x08000b8d   Thumb Code   142  stm32f4xx_exti.o(.text)
    EXTI_StructInit                          0x08000c1b   Thumb Code    16  stm32f4xx_exti.o(.text)
    EXTI_GenerateSWInterrupt                 0x08000c2b   Thumb Code    16  stm32f4xx_exti.o(.text)
    EXTI_GetFlagStatus                       0x08000c3b   Thumb Code    22  stm32f4xx_exti.o(.text)
    EXTI_ClearFlag                           0x08000c51   Thumb Code     8  stm32f4xx_exti.o(.text)
    EXTI_GetITStatus                         0x08000c59   Thumb Code    34  stm32f4xx_exti.o(.text)
    EXTI_ClearITPendingBit                   0x08000c7b   Thumb Code     8  stm32f4xx_exti.o(.text)
    GPIO_DeInit                              0x08000c8d   Thumb Code   220  stm32f4xx_gpio.o(.text)
    GPIO_Init                                0x08000d69   Thumb Code   144  stm32f4xx_gpio.o(.text)
    GPIO_StructInit                          0x08000df9   Thumb Code    18  stm32f4xx_gpio.o(.text)
    GPIO_PinLockConfig                       0x08000e0b   Thumb Code    34  stm32f4xx_gpio.o(.text)
    GPIO_ReadInputDataBit                    0x08000e2d   Thumb Code    18  stm32f4xx_gpio.o(.text)
    GPIO_ReadInputData                       0x08000e3f   Thumb Code     8  stm32f4xx_gpio.o(.text)
    GPIO_ReadOutputDataBit                   0x08000e47   Thumb Code    18  stm32f4xx_gpio.o(.text)
    GPIO_ReadOutputData                      0x08000e59   Thumb Code     8  stm32f4xx_gpio.o(.text)
    GPIO_SetBits                             0x08000e61   Thumb Code     4  stm32f4xx_gpio.o(.text)
    GPIO_ResetBits                           0x08000e65   Thumb Code     4  stm32f4xx_gpio.o(.text)
    GPIO_WriteBit                            0x08000e69   Thumb Code    10  stm32f4xx_gpio.o(.text)
    GPIO_Write                               0x08000e73   Thumb Code     4  stm32f4xx_gpio.o(.text)
    GPIO_ToggleBits                          0x08000e77   Thumb Code     8  stm32f4xx_gpio.o(.text)
    GPIO_PinAFConfig                         0x08000e7f   Thumb Code    70  stm32f4xx_gpio.o(.text)
    I2C_DeInit                               0x08000ee9   Thumb Code    82  stm32f4xx_i2c.o(.text)
    I2C_Init                                 0x08000f3b   Thumb Code   218  stm32f4xx_i2c.o(.text)
    I2C_StructInit                           0x08001015   Thumb Code    30  stm32f4xx_i2c.o(.text)
    I2C_Cmd                                  0x08001033   Thumb Code    24  stm32f4xx_i2c.o(.text)
    I2C_GenerateSTART                        0x0800104b   Thumb Code    24  stm32f4xx_i2c.o(.text)
    I2C_GenerateSTOP                         0x08001063   Thumb Code    24  stm32f4xx_i2c.o(.text)
    I2C_Send7bitAddress                      0x0800107b   Thumb Code    16  stm32f4xx_i2c.o(.text)
    I2C_AcknowledgeConfig                    0x0800108b   Thumb Code    24  stm32f4xx_i2c.o(.text)
    I2C_OwnAddress2Config                    0x080010a3   Thumb Code    22  stm32f4xx_i2c.o(.text)
    I2C_DualAddressCmd                       0x080010b9   Thumb Code    24  stm32f4xx_i2c.o(.text)
    I2C_GeneralCallCmd                       0x080010d1   Thumb Code    24  stm32f4xx_i2c.o(.text)
    I2C_SoftwareResetCmd                     0x080010e9   Thumb Code    22  stm32f4xx_i2c.o(.text)
    I2C_StretchClockCmd                      0x080010ff   Thumb Code    24  stm32f4xx_i2c.o(.text)
    I2C_FastModeDutyCycleConfig              0x08001117   Thumb Code    28  stm32f4xx_i2c.o(.text)
    I2C_NACKPositionConfig                   0x08001133   Thumb Code    28  stm32f4xx_i2c.o(.text)
    I2C_SMBusAlertConfig                     0x0800114f   Thumb Code    28  stm32f4xx_i2c.o(.text)
    I2C_ARPCmd                               0x0800116b   Thumb Code    24  stm32f4xx_i2c.o(.text)
    I2C_SendData                             0x08001183   Thumb Code     4  stm32f4xx_i2c.o(.text)
    I2C_ReceiveData                          0x08001187   Thumb Code     8  stm32f4xx_i2c.o(.text)
    I2C_TransmitPEC                          0x0800118f   Thumb Code    24  stm32f4xx_i2c.o(.text)
    I2C_PECPositionConfig                    0x080011a7   Thumb Code    28  stm32f4xx_i2c.o(.text)
    I2C_CalculatePEC                         0x080011c3   Thumb Code    24  stm32f4xx_i2c.o(.text)
    I2C_GetPEC                               0x080011db   Thumb Code     8  stm32f4xx_i2c.o(.text)
    I2C_DMACmd                               0x080011e3   Thumb Code    24  stm32f4xx_i2c.o(.text)
    I2C_DMALastTransferCmd                   0x080011fb   Thumb Code    24  stm32f4xx_i2c.o(.text)
    I2C_ReadRegister                         0x08001213   Thumb Code    22  stm32f4xx_i2c.o(.text)
    I2C_ITConfig                             0x08001229   Thumb Code    18  stm32f4xx_i2c.o(.text)
    I2C_CheckEvent                           0x0800123b   Thumb Code    42  stm32f4xx_i2c.o(.text)
    I2C_GetLastEvent                         0x08001265   Thumb Code    26  stm32f4xx_i2c.o(.text)
    I2C_GetFlagStatus                        0x0800127f   Thumb Code    58  stm32f4xx_i2c.o(.text)
    I2C_ClearFlag                            0x080012b9   Thumb Code    12  stm32f4xx_i2c.o(.text)
    I2C_GetITStatus                          0x080012c5   Thumb Code    64  stm32f4xx_i2c.o(.text)
    I2C_ClearITPendingBit                    0x08001305   Thumb Code    12  stm32f4xx_i2c.o(.text)
    RCC_DeInit                               0x08001311   Thumb Code    60  stm32f4xx_rcc.o(.text)
    RCC_HSEConfig                            0x0800134d   Thumb Code    14  stm32f4xx_rcc.o(.text)
    RCC_GetFlagStatus                        0x0800135b   Thumb Code    60  stm32f4xx_rcc.o(.text)
    RCC_WaitForHSEStartUp                    0x08001397   Thumb Code    56  stm32f4xx_rcc.o(.text)
    RCC_AdjustHSICalibrationValue            0x080013cf   Thumb Code    20  stm32f4xx_rcc.o(.text)
    RCC_HSICmd                               0x080013e3   Thumb Code     6  stm32f4xx_rcc.o(.text)
    RCC_LSEConfig                            0x080013e9   Thumb Code    46  stm32f4xx_rcc.o(.text)
    RCC_LSICmd                               0x08001417   Thumb Code     6  stm32f4xx_rcc.o(.text)
    RCC_PLLConfig                            0x0800141d   Thumb Code    32  stm32f4xx_rcc.o(.text)
    RCC_PLLCmd                               0x0800143d   Thumb Code     6  stm32f4xx_rcc.o(.text)
    RCC_PLLI2SConfig                         0x08001443   Thumb Code    14  stm32f4xx_rcc.o(.text)
    RCC_PLLI2SCmd                            0x08001451   Thumb Code     6  stm32f4xx_rcc.o(.text)
    RCC_ClockSecuritySystemCmd               0x08001457   Thumb Code     6  stm32f4xx_rcc.o(.text)
    RCC_MCO1Config                           0x0800145d   Thumb Code    28  stm32f4xx_rcc.o(.text)
    RCC_MCO2Config                           0x08001479   Thumb Code    28  stm32f4xx_rcc.o(.text)
    RCC_SYSCLKConfig                         0x08001495   Thumb Code    20  stm32f4xx_rcc.o(.text)
    RCC_GetSYSCLKSource                      0x080014a9   Thumb Code    12  stm32f4xx_rcc.o(.text)
    RCC_HCLKConfig                           0x080014b5   Thumb Code    20  stm32f4xx_rcc.o(.text)
    RCC_PCLK1Config                          0x080014c9   Thumb Code    20  stm32f4xx_rcc.o(.text)
    RCC_PCLK2Config                          0x080014dd   Thumb Code    22  stm32f4xx_rcc.o(.text)
    RCC_GetClocksFreq                        0x080014f3   Thumb Code   222  stm32f4xx_rcc.o(.text)
    RCC_RTCCLKConfig                         0x080015d1   Thumb Code    54  stm32f4xx_rcc.o(.text)
    RCC_RTCCLKCmd                            0x08001607   Thumb Code     8  stm32f4xx_rcc.o(.text)
    RCC_BackupResetCmd                       0x0800160f   Thumb Code     8  stm32f4xx_rcc.o(.text)
    RCC_I2SCLKConfig                         0x08001617   Thumb Code     6  stm32f4xx_rcc.o(.text)
    RCC_AHB1PeriphClockCmd                   0x0800161d   Thumb Code    34  stm32f4xx_rcc.o(.text)
    RCC_AHB2PeriphClockCmd                   0x0800163f   Thumb Code    34  stm32f4xx_rcc.o(.text)
    RCC_AHB3PeriphClockCmd                   0x08001661   Thumb Code    34  stm32f4xx_rcc.o(.text)
    RCC_APB1PeriphClockCmd                   0x08001683   Thumb Code    34  stm32f4xx_rcc.o(.text)
    RCC_APB2PeriphClockCmd                   0x080016a5   Thumb Code    34  stm32f4xx_rcc.o(.text)
    RCC_AHB1PeriphResetCmd                   0x080016c7   Thumb Code    34  stm32f4xx_rcc.o(.text)
    RCC_AHB2PeriphResetCmd                   0x080016e9   Thumb Code    72  stm32f4xx_rcc.o(.text)
    RCC_AHB3PeriphResetCmd                   0x08001731   Thumb Code    34  stm32f4xx_rcc.o(.text)
    RCC_APB1PeriphResetCmd                   0x08001753   Thumb Code    34  stm32f4xx_rcc.o(.text)
    RCC_APB2PeriphResetCmd                   0x08001775   Thumb Code    34  stm32f4xx_rcc.o(.text)
    RCC_AHB1PeriphClockLPModeCmd             0x08001797   Thumb Code    34  stm32f4xx_rcc.o(.text)
    RCC_AHB2PeriphClockLPModeCmd             0x080017b9   Thumb Code    34  stm32f4xx_rcc.o(.text)
    RCC_AHB3PeriphClockLPModeCmd             0x080017db   Thumb Code    34  stm32f4xx_rcc.o(.text)
    RCC_APB1PeriphClockLPModeCmd             0x080017fd   Thumb Code    34  stm32f4xx_rcc.o(.text)
    RCC_APB2PeriphClockLPModeCmd             0x0800181f   Thumb Code    34  stm32f4xx_rcc.o(.text)
    RCC_ITConfig                             0x08001841   Thumb Code    34  stm32f4xx_rcc.o(.text)
    RCC_ClearFlag                            0x08001863   Thumb Code    18  stm32f4xx_rcc.o(.text)
    RCC_GetITStatus                          0x08001875   Thumb Code    22  stm32f4xx_rcc.o(.text)
    RCC_ClearITPendingBit                    0x0800188b   Thumb Code     8  stm32f4xx_rcc.o(.text)
    SPI_I2S_DeInit                           0x08001899   Thumb Code    76  stm32f4xx_spi.o(.text)
    SPI_Init                                 0x080018e5   Thumb Code    60  stm32f4xx_spi.o(.text)
    I2S_Init                                 0x08001921   Thumb Code   346  stm32f4xx_spi.o(.text)
    SPI_StructInit                           0x08001a7b   Thumb Code    24  stm32f4xx_spi.o(.text)
    I2S_StructInit                           0x08001a93   Thumb Code    20  stm32f4xx_spi.o(.text)
    SPI_Cmd                                  0x08001aa7   Thumb Code    24  stm32f4xx_spi.o(.text)
    I2S_Cmd                                  0x08001abf   Thumb Code    24  stm32f4xx_spi.o(.text)
    SPI_DataSizeConfig                       0x08001ad7   Thumb Code    18  stm32f4xx_spi.o(.text)
    SPI_BiDirectionalLineConfig              0x08001ae9   Thumb Code    28  stm32f4xx_spi.o(.text)
    SPI_NSSInternalSoftwareConfig            0x08001b05   Thumb Code    30  stm32f4xx_spi.o(.text)
    SPI_SSOutputCmd                          0x08001b23   Thumb Code    24  stm32f4xx_spi.o(.text)
    SPI_TIModeCmd                            0x08001b3b   Thumb Code    24  stm32f4xx_spi.o(.text)
    I2S_FullDuplexConfig                     0x08001b53   Thumb Code    80  stm32f4xx_spi.o(.text)
    SPI_I2S_ReceiveData                      0x08001ba3   Thumb Code     6  stm32f4xx_spi.o(.text)
    SPI_I2S_SendData                         0x08001ba9   Thumb Code     4  stm32f4xx_spi.o(.text)
    SPI_CalculateCRC                         0x08001bad   Thumb Code    24  stm32f4xx_spi.o(.text)
    SPI_TransmitCRC                          0x08001bc5   Thumb Code    10  stm32f4xx_spi.o(.text)
    SPI_GetCRC                               0x08001bcf   Thumb Code    16  stm32f4xx_spi.o(.text)
    SPI_GetCRCPolynomial                     0x08001bdf   Thumb Code     6  stm32f4xx_spi.o(.text)
    SPI_I2S_DMACmd                           0x08001be5   Thumb Code    18  stm32f4xx_spi.o(.text)
    SPI_I2S_ITConfig                         0x08001bf7   Thumb Code    32  stm32f4xx_spi.o(.text)
    SPI_I2S_GetFlagStatus                    0x08001c17   Thumb Code    18  stm32f4xx_spi.o(.text)
    SPI_I2S_ClearFlag                        0x08001c29   Thumb Code     6  stm32f4xx_spi.o(.text)
    SPI_I2S_GetITStatus                      0x08001c2f   Thumb Code    52  stm32f4xx_spi.o(.text)
    SPI_I2S_ClearITPendingBit                0x08001c63   Thumb Code    20  stm32f4xx_spi.o(.text)
    SYSCFG_DeInit                            0x08001c8d   Thumb Code    22  stm32f4xx_syscfg.o(.text)
    SYSCFG_MemoryRemapConfig                 0x08001ca3   Thumb Code     6  stm32f4xx_syscfg.o(.text)
    SYSCFG_EXTILineConfig                    0x08001ca9   Thumb Code    66  stm32f4xx_syscfg.o(.text)
    SYSCFG_ETH_MediaInterfaceConfig          0x08001ceb   Thumb Code     6  stm32f4xx_syscfg.o(.text)
    SYSCFG_CompensationCellCmd               0x08001cf1   Thumb Code     6  stm32f4xx_syscfg.o(.text)
    SYSCFG_GetCompensationCellStatus         0x08001cf7   Thumb Code    22  stm32f4xx_syscfg.o(.text)
    USBD_DeInit                              0x080020e5   Thumb Code     6  usbd_core.o(.text)
    USBD_Init                                0x080020eb   Thumb Code    66  usbd_core.o(.text)
    USBD_SetCfg                              0x0800234b   Thumb Code    30  usbd_core.o(.text)
    USBD_ClrCfg                              0x08002369   Thumb Code    22  usbd_core.o(.text)
    USBD_CtlSendData                         0x080023a3   Thumb Code    46  usbd_ioreq.o(.text)
    USBD_CtlContinueSendData                 0x080023d1   Thumb Code    30  usbd_ioreq.o(.text)
    USBD_CtlPrepareRx                        0x080023ef   Thumb Code    46  usbd_ioreq.o(.text)
    USBD_CtlContinueRx                       0x0800241d   Thumb Code    30  usbd_ioreq.o(.text)
    USBD_CtlSendStatus                       0x0800243b   Thumb Code    36  usbd_ioreq.o(.text)
    USBD_CtlReceiveStatus                    0x0800245f   Thumb Code    36  usbd_ioreq.o(.text)
    USBD_GetRxCount                          0x08002483   Thumb Code    20  usbd_ioreq.o(.text)
    USBD_CtlError                            0x08002499   Thumb Code    56  usbd_req.o(.text)
    USBD_StdDevReq                           0x08002891   Thumb Code   114  usbd_req.o(.text)
    USBD_StdItfReq                           0x08002903   Thumb Code    76  usbd_req.o(.text)
    USBD_StdEPReq                            0x0800294f   Thumb Code   358  usbd_req.o(.text)
    USBD_ParseSetupRequest                   0x08002ab5   Thumb Code    72  usbd_req.o(.text)
    USBD_GetString                           0x08002b11   Thumb Code    82  usbd_req.o(.text)
    USB_OTG_WritePacket                      0x08002c01   Thumb Code    64  usb_core.o(.text)
    USB_OTG_ReadPacket                       0x08002c41   Thumb Code    40  usb_core.o(.text)
    USB_OTG_SelectCore                       0x08002c69   Thumb Code   204  usb_core.o(.text)
    USB_OTG_CoreInit                         0x08002d35   Thumb Code   462  usb_core.o(.text)
    USB_OTG_EnableGlobalInt                  0x08002f03   Thumb Code    34  usb_core.o(.text)
    USB_OTG_DisableGlobalInt                 0x08002f25   Thumb Code    34  usb_core.o(.text)
    USB_OTG_FlushTxFifo                      0x08002f47   Thumb Code    90  usb_core.o(.text)
    USB_OTG_FlushRxFifo                      0x08002fa1   Thumb Code    70  usb_core.o(.text)
    USB_OTG_SetCurrentMode                   0x08002fe7   Thumb Code    78  usb_core.o(.text)
    USB_OTG_GetMode                          0x08003035   Thumb Code    12  usb_core.o(.text)
    USB_OTG_IsDeviceMode                     0x08003041   Thumb Code    22  usb_core.o(.text)
    USB_OTG_IsHostMode                       0x08003057   Thumb Code    20  usb_core.o(.text)
    USB_OTG_ReadCoreItr                      0x0800306b   Thumb Code    16  usb_core.o(.text)
    USB_OTG_ReadOtgItr                       0x0800307b   Thumb Code     8  usb_core.o(.text)
    USB_OTG_InitDevSpeed                     0x08003083   Thumb Code    24  usb_core.o(.text)
    USB_OTG_EnableDevInt                     0x0800309b   Thumb Code   152  usb_core.o(.text)
    USB_OTG_CoreInitDev                      0x08003133   Thumb Code   522  usb_core.o(.text)
    USB_OTG_GetDeviceSpeed                   0x0800333d   Thumb Code    52  usb_core.o(.text)
    USB_OTG_EP0Activate                      0x08003371   Thumb Code   112  usb_core.o(.text)
    USB_OTG_EPActivate                       0x080033e1   Thumb Code   152  usb_core.o(.text)
    USB_OTG_EPDeactivate                     0x08003479   Thumb Code    94  usb_core.o(.text)
    USB_OTG_EPStartXfer                      0x080034d7   Thumb Code   506  usb_core.o(.text)
    USB_OTG_EP0StartXfer                     0x080036d1   Thumb Code   342  usb_core.o(.text)
    USB_OTG_EPSetStall                       0x08003827   Thumb Code   100  usb_core.o(.text)
    USB_OTG_EPClearStall                     0x0800388b   Thumb Code    80  usb_core.o(.text)
    USB_OTG_ReadDevAllOutEp_itr              0x080038db   Thumb Code    16  usb_core.o(.text)
    USB_OTG_ReadDevOutEP_itr                 0x080038eb   Thumb Code    20  usb_core.o(.text)
    USB_OTG_ReadDevAllInEPItr                0x080038ff   Thumb Code    16  usb_core.o(.text)
    USB_OTG_EP0_OutStart                     0x0800390f   Thumb Code    98  usb_core.o(.text)
    USB_OTG_ActiveRemoteWakeup               0x08003971   Thumb Code   106  usb_core.o(.text)
    USB_OTG_UngateClock                      0x080039db   Thumb Code    54  usb_core.o(.text)
    USB_OTG_StopDevice                       0x08003a11   Thumb Code    82  usb_core.o(.text)
    USB_OTG_GetEPStatus                      0x08003a63   Thumb Code   106  usb_core.o(.text)
    USB_OTG_SetEPStatus                      0x08003acd   Thumb Code   282  usb_core.o(.text)
    DCD_Init                                 0x08003be7   Thumb Code   156  usb_dcd.o(.text)
    DCD_EP_Open                              0x08003c83   Thumb Code   104  usb_dcd.o(.text)
    DCD_EP_Close                             0x08003ceb   Thumb Code    74  usb_dcd.o(.text)
    DCD_EP_PrepareRx                         0x08003d35   Thumb Code    82  usb_dcd.o(.text)
    DCD_EP_Tx                                0x08003d87   Thumb Code    78  usb_dcd.o(.text)
    DCD_EP_Stall                             0x08003dd5   Thumb Code    72  usb_dcd.o(.text)
    DCD_EP_ClrStall                          0x08003e1d   Thumb Code    72  usb_dcd.o(.text)
    DCD_EP_Flush                             0x08003e65   Thumb Code    36  usb_dcd.o(.text)
    DCD_EP_SetAddress                        0x08003e89   Thumb Code    28  usb_dcd.o(.text)
    DCD_DevConnect                           0x08003ea5   Thumb Code    32  usb_dcd.o(.text)
    DCD_DevDisconnect                        0x08003ec5   Thumb Code    34  usb_dcd.o(.text)
    DCD_GetEPStatus                          0x08003ee7   Thumb Code    64  usb_dcd.o(.text)
    DCD_SetEPStatus                          0x08003f27   Thumb Code    62  usb_dcd.o(.text)
    USBD_OTG_ISR_Handler                     0x08004651   Thumb Code   224  usb_dcd_int.o(.text)
    main                                     0x08004735   Thumb Code    22  main.o(.text)
    Delay                                    0x0800474b   Thumb Code    20  main.o(.text)
    TimingDelay_Decrement                    0x0800475f   Thumb Code    18  main.o(.text)
    EVAL_AUDIO_TransferComplete_CallBack     0x08004771   Thumb Code     2  main.o(.text)
    NMI_Handler                              0x08004789   Thumb Code     2  stm32f4xx_it.o(.text)
    HardFault_Handler                        0x0800478b   Thumb Code     4  stm32f4xx_it.o(.text)
    MemManage_Handler                        0x0800478f   Thumb Code     4  stm32f4xx_it.o(.text)
    BusFault_Handler                         0x08004793   Thumb Code     4  stm32f4xx_it.o(.text)
    UsageFault_Handler                       0x08004797   Thumb Code     4  stm32f4xx_it.o(.text)
    SVC_Handler                              0x0800479b   Thumb Code     2  stm32f4xx_it.o(.text)
    DebugMon_Handler                         0x0800479d   Thumb Code     2  stm32f4xx_it.o(.text)
    PendSV_Handler                           0x0800479f   Thumb Code     2  stm32f4xx_it.o(.text)
    SysTick_Handler                          0x080047a1   Thumb Code     2  stm32f4xx_it.o(.text)
    OTG_FS_WKUP_IRQHandler                   0x080047a3   Thumb Code    40  stm32f4xx_it.o(.text)
    OTG_FS_IRQHandler                        0x080047cb   Thumb Code    10  stm32f4xx_it.o(.text)
    USB_OTG_BSP_Init                         0x080047dd   Thumb Code   160  usb_bsp.o(.text)
    USB_OTG_BSP_EnableInterrupt              0x0800487d   Thumb Code    44  usb_bsp.o(.text)
    USB_OTG_BSP_uDelay                       0x080048a9   Thumb Code    30  usb_bsp.o(.text)
    USB_OTG_BSP_mDelay                       0x080048c7   Thumb Code    18  usb_bsp.o(.text)
    USBD_USR_DeviceDescriptor                0x080048dd   Thumb Code    10  usbd_desc.o(.text)
    USBD_USR_LangIDStrDescriptor             0x080048e7   Thumb Code    10  usbd_desc.o(.text)
    USBD_USR_ProductStrDescriptor            0x080048f1   Thumb Code    34  usbd_desc.o(.text)
    USBD_USR_ManufacturerStrDescriptor       0x08004913   Thumb Code    20  usbd_desc.o(.text)
    USBD_USR_SerialStrDescriptor             0x08004927   Thumb Code    34  usbd_desc.o(.text)
    USBD_USR_ConfigStrDescriptor             0x08004949   Thumb Code    34  usbd_desc.o(.text)
    USBD_USR_InterfaceStrDescriptor          0x0800496b   Thumb Code    34  usbd_desc.o(.text)
    USBD_USR_Init                            0x08004a35   Thumb Code    90  usbd_usr.o(.text)
    USBD_USR_DeviceReset                     0x08004a8f   Thumb Code    18  usbd_usr.o(.text)
    USBD_USR_DeviceConfigured                0x08004aa1   Thumb Code     2  usbd_usr.o(.text)
    USBD_USR_DeviceConnected                 0x08004aa3   Thumb Code     2  usbd_usr.o(.text)
    USBD_USR_DeviceDisconnected              0x08004aa5   Thumb Code     2  usbd_usr.o(.text)
    USBD_USR_DeviceSuspended                 0x08004aa7   Thumb Code     2  usbd_usr.o(.text)
    USBD_USR_DeviceResumed                   0x08004aa9   Thumb Code     2  usbd_usr.o(.text)
    STM_EVAL_LEDInit                         0x08004ab9   Thumb Code    62  stm32f4_discovery.o(.text)
    STM_EVAL_LEDOn                           0x08004af7   Thumb Code    16  stm32f4_discovery.o(.text)
    STM_EVAL_LEDOff                          0x08004b07   Thumb Code    16  stm32f4_discovery.o(.text)
    STM_EVAL_LEDToggle                       0x08004b17   Thumb Code    26  stm32f4_discovery.o(.text)
    STM_EVAL_PBInit                          0x08004b31   Thumb Code   140  stm32f4_discovery.o(.text)
    STM_EVAL_PBGetState                      0x08004bbd   Thumb Code    22  stm32f4_discovery.o(.text)
    EVAL_AUDIO_SetAudioInterface             0x08004bfd   Thumb Code   156  stm32f4_discovery_audio_codec.o(.text)
    Codec_TIMEOUT_UserCallback               0x08004d35   Thumb Code     4  stm32f4_discovery_audio_codec.o(.text)
    EVAL_AUDIO_Init                          0x080052e3   Thumb Code    58  stm32f4_discovery_audio_codec.o(.text)
    EVAL_AUDIO_DeInit                        0x080053d7   Thumb Code    14  stm32f4_discovery_audio_codec.o(.text)
    Audio_MAL_Play                           0x080053e5   Thumb Code   242  stm32f4_discovery_audio_codec.o(.text)
    EVAL_AUDIO_Play                          0x080054db   Thumb Code   110  stm32f4_discovery_audio_codec.o(.text)
    EVAL_AUDIO_PauseResume                   0x080055f9   Thumb Code    28  stm32f4_discovery_audio_codec.o(.text)
    EVAL_AUDIO_Stop                          0x08005689   Thumb Code    32  stm32f4_discovery_audio_codec.o(.text)
    EVAL_AUDIO_VolumeCtl                     0x080056a9   Thumb Code    32  stm32f4_discovery_audio_codec.o(.text)
    EVAL_AUDIO_Mute                          0x080056c9   Thumb Code    12  stm32f4_discovery_audio_codec.o(.text)
    DMA1_Stream7_IRQHandler                  0x080056df   Thumb Code     8  stm32f4_discovery_audio_codec.o(.text)
    DMA1_Stream0_IRQHandler                  0x080056e7   Thumb Code     8  stm32f4_discovery_audio_codec.o(.text)
    EVAL_AUDIO_GetSampleCallBack             0x080056ef   Thumb Code   106  stm32f4_discovery_audio_codec.o(.text)
    SPI3_IRQHandler                          0x08005759   Thumb Code    66  stm32f4_discovery_audio_codec.o(.text)
    DAC_Config                               0x0800579b   Thumb Code    76  stm32f4_discovery_audio_codec.o(.text)
    __use_two_region_memory                  0x08005831   Thumb Code     2  heapauxi.o(.text)
    __rt_heap_escrow$2region                 0x08005833   Thumb Code     2  heapauxi.o(.text)
    __rt_heap_expand$2region                 0x08005835   Thumb Code     2  heapauxi.o(.text)
    __user_setup_stackheap                   0x08005837   Thumb Code    74  sys_stackheap_outer.o(.text)
    exit                                     0x08005881   Thumb Code    12  exit.o(.text)
    __user_libspace                          0x0800588d   Thumb Code     8  libspace.o(.text)
    __user_perproc_libspace                  0x0800588d   Thumb Code     0  libspace.o(.text)
    __user_perthread_libspace                0x0800588d   Thumb Code     0  libspace.o(.text)
    _sys_exit                                0x08005895   Thumb Code     8  sys_exit.o(.text)
    __I$use$semihosting                      0x080058a1   Thumb Code     0  use_no_semi.o(.text)
    __use_no_semihosting_swi                 0x080058a1   Thumb Code     2  use_no_semi.o(.text)
    __semihosting_library_function           0x080058a3   Thumb Code     0  indicate_semi.o(.text)
    GPIO_PIN                                 0x080058a4   Data           8  stm32f4_discovery.o(.constdata)
    GPIO_CLK                                 0x080058ac   Data          16  stm32f4_discovery.o(.constdata)
    BUTTON_PIN                               0x080058bc   Data           2  stm32f4_discovery.o(.constdata)
    BUTTON_CLK                               0x080058c0   Data           4  stm32f4_discovery.o(.constdata)
    BUTTON_EXTI_LINE                         0x080058c4   Data           2  stm32f4_discovery.o(.constdata)
    BUTTON_PORT_SOURCE                       0x080058c6   Data           1  stm32f4_discovery.o(.constdata)
    BUTTON_PIN_SOURCE                        0x080058c7   Data           1  stm32f4_discovery.o(.constdata)
    BUTTON_IRQn                              0x080058c8   Data           1  stm32f4_discovery.o(.constdata)
    Region$$Table$$Base                      0x080058cc   Number         0  anon$$obj.o(Region$$Table)
    Region$$Table$$Limit                     0x080058ec   Number         0  anon$$obj.o(Region$$Table)
    SystemCoreClock                          0x20000000   Data           4  system_stm32f4xx.o(.data)
    AHBPrescTable                            0x20000004   Data          16  system_stm32f4xx.o(.data)
    IsocOutWrPtr                             0x20000024   Data           4  usbd_audio_core.o(.data)
    IsocOutRdPtr                             0x20000028   Data           4  usbd_audio_core.o(.data)
    AudioCtlCmd                              0x2000002c   Data           1  usbd_audio_core.o(.data)
    AudioCtlLen                              0x20000030   Data           4  usbd_audio_core.o(.data)
    AudioCtlUnit                             0x20000034   Data           1  usbd_audio_core.o(.data)
    AUDIO_cb                                 0x20000040   Data          44  usbd_audio_core.o(.data)
    AUDIO_OUT_fops                           0x200000dc   Data          28  usbd_audio_out_if.o(.data)
    USBD_DCD_INT_cb                          0x20000100   Data          44  usbd_core.o(.data)
    USBD_DCD_INT_fops                        0x2000012c   Data           4  usbd_core.o(.data)
    USBD_ep_status                           0x20000130   Data           4  usbd_req.o(.data)
    USBD_default_cfg                         0x20000134   Data           4  usbd_req.o(.data)
    USBD_cfg_status                          0x20000138   Data           4  usbd_req.o(.data)
    PrescalerValue                           0x20000140   Data           2  main.o(.data)
    UserButtonPressed                        0x20000142   Data           1  main.o(.data)
    TimingDelay                              0x20000144   Data           4  main.o(.data)
    Buffer                                   0x20000148   Data           6  main.o(.data)
    USR_desc                                 0x20000150   Data          28  usbd_desc.o(.data)
    USBD_DeviceDesc                          0x2000016c   Data          18  usbd_desc.o(.data)
    USBD_DeviceQualifierDesc                 0x2000017e   Data          10  usbd_desc.o(.data)
    USBD_LangIDDesc                          0x20000188   Data           4  usbd_desc.o(.data)
    USR_cb                                   0x2000018c   Data          28  usbd_usr.o(.data)
    GPIO_PORT                                0x200001a8   Data          16  stm32f4_discovery.o(.data)
    BUTTON_PORT                              0x200001b8   Data           4  stm32f4_discovery.o(.data)
    NVIC_InitStructure                       0x200001bc   Data           4  stm32f4_discovery.o(.data)
    AudioTotalSize                           0x200001c0   Data           4  stm32f4_discovery_audio_codec.o(.data)
    AudioRemSize                             0x200001c4   Data           4  stm32f4_discovery_audio_codec.o(.data)
    CODECTimeout                             0x200001c8   Data           4  stm32f4_discovery_audio_codec.o(.data)
    OutputDev                                0x200001cc   Data           1  stm32f4_discovery_audio_codec.o(.data)
    CurrAudioInterface                       0x200001d0   Data           4  stm32f4_discovery_audio_codec.o(.data)
    AUDIO_MAL_DMA_CLOCK                      0x200001d4   Data           4  stm32f4_discovery_audio_codec.o(.data)
    AUDIO_MAL_DMA_STREAM                     0x200001d8   Data           4  stm32f4_discovery_audio_codec.o(.data)
    AUDIO_MAL_DMA_DREG                       0x200001dc   Data           4  stm32f4_discovery_audio_codec.o(.data)
    AUDIO_MAL_DMA_CHANNEL                    0x200001e0   Data           4  stm32f4_discovery_audio_codec.o(.data)
    AUDIO_MAL_DMA_IRQ                        0x200001e4   Data           4  stm32f4_discovery_audio_codec.o(.data)
    AUDIO_MAL_DMA_FLAG_TC                    0x200001e8   Data           4  stm32f4_discovery_audio_codec.o(.data)
    AUDIO_MAL_DMA_FLAG_HT                    0x200001ec   Data           4  stm32f4_discovery_audio_codec.o(.data)
    AUDIO_MAL_DMA_FLAG_FE                    0x200001f0   Data           4  stm32f4_discovery_audio_codec.o(.data)
    AUDIO_MAL_DMA_FLAG_TE                    0x200001f4   Data           4  stm32f4_discovery_audio_codec.o(.data)
    AUDIO_MAL_DMA_FLAG_DME                   0x200001f8   Data           4  stm32f4_discovery_audio_codec.o(.data)
    CurrentPos                               0x20000200   Data           4  stm32f4_discovery_audio_codec.o(.data)
    dac_play_ptr                             0x20000204   Data           4  stm32f4_discovery_audio_codec.o(.data)
    dac_play_size                            0x20000208   Data           2  stm32f4_discovery_audio_codec.o(.data)
    dac_play_cnt                             0x2000020a   Data           2  stm32f4_discovery_audio_codec.o(.data)
    IsocOutBuff                              0x2000020c   Data        1536  usbd_audio_core.o(.bss)
    AudioCtl                                 0x2000080c   Data          64  usbd_audio_core.o(.bss)
    USBD_StrDesc                             0x2000084c   Data         200  usbd_req.o(.bss)
    USB_OTG_dev                              0x20000914   Data        1520  main.o(.bss)
    DMA_InitStructure                        0x20000f04   Data          60  stm32f4_discovery_audio_codec.o(.bss)
    AUDIO_MAL_DMA_InitStructure              0x20000f40   Data          60  stm32f4_discovery_audio_codec.o(.bss)
    __libspace_start                         0x20000f7c   Data          96  libspace.o(.bss)
    __temporary_stack_top$libspace           0x20000fdc   Data           0  libspace.o(.bss)



==============================================================================

Memory Map of the image

  Image Entry point : 0x08000189

  Load Region LR_IROM1 (Base: 0x08000000, Size: 0x00005af8, Max: 0x00100000, ABSOLUTE, COMPRESSED[0x00005a2c])

    Execution Region ER_IROM1 (Base: 0x08000000, Size: 0x000058ec, Max: 0x00100000, ABSOLUTE)

    Base Addr    Size         Type   Attr      Idx    E Section Name        Object

    0x08000000   0x00000188   Data   RO            3    RESET               startup_stm32f40_41xxx.o
    0x08000188   0x00000008   Code   RO         1195  * !!!main             c_w.l(__main.o)
    0x08000190   0x00000034   Code   RO         1351    !!!scatter          c_w.l(__scatter.o)
    0x080001c4   0x0000005a   Code   RO         1349    !!dczerorl2         c_w.l(__dczerorl2.o)
    0x0800021e   0x00000002   PAD
    0x08000220   0x0000001c   Code   RO         1353    !!handler_zi        c_w.l(__scatter_zi.o)
    0x0800023c   0x00000002   Code   RO         1222    .ARM.Collect$$libinit$$00000000  c_w.l(libinit.o)
    0x0800023e   0x00000000   Code   RO         1229    .ARM.Collect$$libinit$$00000002  c_w.l(libinit2.o)
    0x0800023e   0x00000000   Code   RO         1232    .ARM.Collect$$libinit$$00000008  c_w.l(libinit2.o)
    0x0800023e   0x00000000   Code   RO         1234    .ARM.Collect$$libinit$$0000000A  c_w.l(libinit2.o)
    0x0800023e   0x00000000   Code   RO         1236    .ARM.Collect$$libinit$$0000000C  c_w.l(libinit2.o)
    0x0800023e   0x00000000   Code   RO         1239    .ARM.Collect$$libinit$$0000000F  c_w.l(libinit2.o)
    0x0800023e   0x00000000   Code   RO         1241    .ARM.Collect$$libinit$$00000011  c_w.l(libinit2.o)
    0x0800023e   0x00000000   Code   RO         1243    .ARM.Collect$$libinit$$00000013  c_w.l(libinit2.o)
    0x0800023e   0x00000000   Code   RO         1245    .ARM.Collect$$libinit$$00000015  c_w.l(libinit2.o)
    0x0800023e   0x00000000   Code   RO         1247    .ARM.Collect$$libinit$$00000017  c_w.l(libinit2.o)
    0x0800023e   0x00000000   Code   RO         1249    .ARM.Collect$$libinit$$00000019  c_w.l(libinit2.o)
    0x0800023e   0x00000000   Code   RO         1251    .ARM.Collect$$libinit$$0000001B  c_w.l(libinit2.o)
    0x0800023e   0x00000000   Code   RO         1253    .ARM.Collect$$libinit$$0000001D  c_w.l(libinit2.o)
    0x0800023e   0x00000000   Code   RO         1255    .ARM.Collect$$libinit$$0000001F  c_w.l(libinit2.o)
    0x0800023e   0x00000000   Code   RO         1257    .ARM.Collect$$libinit$$00000021  c_w.l(libinit2.o)
    0x0800023e   0x00000000   Code   RO         1259    .ARM.Collect$$libinit$$00000023  c_w.l(libinit2.o)
    0x0800023e   0x00000000   Code   RO         1263    .ARM.Collect$$libinit$$0000002A  c_w.l(libinit2.o)
    0x0800023e   0x00000000   Code   RO         1265    .ARM.Collect$$libinit$$0000002C  c_w.l(libinit2.o)
    0x0800023e   0x00000000   Code   RO         1267    .ARM.Collect$$libinit$$0000002E  c_w.l(libinit2.o)
    0x0800023e   0x00000000   Code   RO         1269    .ARM.Collect$$libinit$$00000030  c_w.l(libinit2.o)
    0x0800023e   0x00000002   Code   RO         1270    .ARM.Collect$$libinit$$00000031  c_w.l(libinit2.o)
    0x08000240   0x00000002   Code   RO         1290    .ARM.Collect$$libshutdown$$00000000  c_w.l(libshutdown.o)
    0x08000242   0x00000000   Code   RO         1304    .ARM.Collect$$libshutdown$$00000003  c_w.l(libshutdown2.o)
    0x08000242   0x00000000   Code   RO         1307    .ARM.Collect$$libshutdown$$00000006  c_w.l(libshutdown2.o)
    0x08000242   0x00000000   Code   RO         1310    .ARM.Collect$$libshutdown$$00000009  c_w.l(libshutdown2.o)
    0x08000242   0x00000000   Code   RO         1312    .ARM.Collect$$libshutdown$$0000000B  c_w.l(libshutdown2.o)
    0x08000242   0x00000000   Code   RO         1315    .ARM.Collect$$libshutdown$$0000000E  c_w.l(libshutdown2.o)
    0x08000242   0x00000002   Code   RO         1316    .ARM.Collect$$libshutdown$$0000000F  c_w.l(libshutdown2.o)
    0x08000244   0x00000000   Code   RO         1197    .ARM.Collect$$rtentry$$00000000  c_w.l(rtentry.o)
    0x08000244   0x00000000   Code   RO         1199    .ARM.Collect$$rtentry$$00000002  c_w.l(rtentry2.o)
    0x08000244   0x00000006   Code   RO         1211    .ARM.Collect$$rtentry$$00000004  c_w.l(rtentry4.o)
    0x0800024a   0x00000000   Code   RO         1201    .ARM.Collect$$rtentry$$00000009  c_w.l(rtentry2.o)
    0x0800024a   0x00000004   Code   RO         1202    .ARM.Collect$$rtentry$$0000000A  c_w.l(rtentry2.o)
    0x0800024e   0x00000000   Code   RO         1204    .ARM.Collect$$rtentry$$0000000C  c_w.l(rtentry2.o)
    0x0800024e   0x00000008   Code   RO         1205    .ARM.Collect$$rtentry$$0000000D  c_w.l(rtentry2.o)
    0x08000256   0x00000002   Code   RO         1226    .ARM.Collect$$rtexit$$00000000  c_w.l(rtexit.o)
    0x08000258   0x00000000   Code   RO         1272    .ARM.Collect$$rtexit$$00000002  c_w.l(rtexit2.o)
    0x08000258   0x00000004   Code   RO         1273    .ARM.Collect$$rtexit$$00000003  c_w.l(rtexit2.o)
    0x0800025c   0x00000006   Code   RO         1274    .ARM.Collect$$rtexit$$00000004  c_w.l(rtexit2.o)
    0x08000262   0x00000002   PAD
    0x08000264   0x00000040   Code   RO            4    .text               startup_stm32f40_41xxx.o
    0x080002a4   0x00000234   Code   RO           12    .text               system_stm32f4xx.o
    0x080004d8   0x000000e4   Code   RO          139    .text               misc.o
    0x080005bc   0x00000210   Code   RO          303    .text               stm32f4xx_dac.o
    0x080007cc   0x000003a4   Code   RO          363    .text               stm32f4xx_dma.o
    0x08000b70   0x0000011c   Code   RO          383    .text               stm32f4xx_exti.o
    0x08000c8c   0x0000025c   Code   RO          443    .text               stm32f4xx_gpio.o
    0x08000ee8   0x00000428   Code   RO          523    .text               stm32f4xx_i2c.o
    0x08001310   0x00000588   Code   RO          583    .text               stm32f4xx_rcc.o
    0x08001898   0x000003f4   Code   RO          665    .text               stm32f4xx_spi.o
    0x08001c8c   0x0000008c   Code   RO          685    .text               stm32f4xx_syscfg.o
    0x08001d18   0x00000284   Code   RO          765    .text               usbd_audio_core.o
    0x08001f9c   0x00000148   Code   RO          832    .text               usbd_audio_out_if.o
    0x080020e4   0x000002be   Code   RO          864    .text               usbd_core.o
    0x080023a2   0x000000f4   Code   RO          893    .text               usbd_ioreq.o
    0x08002496   0x00000002   PAD
    0x08002498   0x000006d0   Code   RO          913    .text               usbd_req.o
    0x08002b68   0x0000107e   Code   RO          941    .text               usb_core.o
    0x08003be6   0x0000037e   Code   RO          961    .text               usb_dcd.o
    0x08003f64   0x000007d0   Code   RO          981    .text               usb_dcd_int.o
    0x08004734   0x00000054   Code   RO         1005    .text               main.o
    0x08004788   0x00000054   Code   RO         1043    .text               stm32f4xx_it.o
    0x080047dc   0x00000100   Code   RO         1067    .text               usb_bsp.o
    0x080048dc   0x00000158   Code   RO         1087    .text               usbd_desc.o
    0x08004a34   0x00000084   Code   RO         1114    .text               usbd_usr.o
    0x08004ab8   0x00000144   Code   RO         1145    .text               stm32f4_discovery.o
    0x08004bfc   0x00000c34   Code   RO         1169    .text               stm32f4_discovery_audio_codec.o
    0x08005830   0x00000006   Code   RO         1193    .text               c_w.l(heapauxi.o)
    0x08005836   0x0000004a   Code   RO         1213    .text               c_w.l(sys_stackheap_outer.o)
    0x08005880   0x0000000c   Code   RO         1215    .text               c_w.l(exit.o)
    0x0800588c   0x00000008   Code   RO         1223    .text               c_w.l(libspace.o)
    0x08005894   0x0000000c   Code   RO         1282    .text               c_w.l(sys_exit.o)
    0x080058a0   0x00000002   Code   RO         1293    .text               c_w.l(use_no_semi.o)
    0x080058a2   0x00000000   Code   RO         1295    .text               c_w.l(indicate_semi.o)
    0x080058a2   0x00000002   PAD
    0x080058a4   0x00000025   Data   RO         1146    .constdata          stm32f4_discovery.o
    0x080058c9   0x00000003   PAD
    0x080058cc   0x00000020   Data   RO         1347    Region$$Table       anon$$obj.o


    Execution Region RW_IRAM1 (Base: 0x20000000, Size: 0x000015e0, Max: 0x00020000, ABSOLUTE, COMPRESSED[0x00000140])

    Base Addr    Size         Type   Attr      Idx    E Section Name        Object

    0x20000000   0x00000014   Data   RW           13    .data               system_stm32f4xx.o
    0x20000014   0x00000010   Data   RW          584    .data               stm32f4xx_rcc.o
    0x20000024   0x000000b5   Data   RW          767    .data               usbd_audio_core.o
    0x200000d9   0x00000003   PAD
    0x200000dc   0x00000024   Data   RW          833    .data               usbd_audio_out_if.o
    0x20000100   0x00000030   Data   RW          865    .data               usbd_core.o
    0x20000130   0x0000000d   Data   RW          915    .data               usbd_req.o
    0x2000013d   0x00000003   PAD
    0x20000140   0x0000000e   Data   RW         1007    .data               main.o
    0x2000014e   0x00000002   PAD
    0x20000150   0x0000003c   Data   RW         1088    .data               usbd_desc.o
    0x2000018c   0x0000001c   Data   RW         1115    .data               usbd_usr.o
    0x200001a8   0x00000018   Data   RW         1147    .data               stm32f4_discovery.o
    0x200001c0   0x0000004c   Data   RW         1171    .data               stm32f4_discovery_audio_codec.o
    0x2000020c   0x00000640   Zero   RW          766    .bss                usbd_audio_core.o
    0x2000084c   0x000000c8   Zero   RW          914    .bss                usbd_req.o
    0x20000914   0x000005f0   Zero   RW         1006    .bss                main.o
    0x20000f04   0x00000078   Zero   RW         1170    .bss                stm32f4_discovery_audio_codec.o
    0x20000f7c   0x00000060   Zero   RW         1224    .bss                c_w.l(libspace.o)
    0x20000fdc   0x00000004   PAD
    0x20000fe0   0x00000200   Zero   RW            2    HEAP                startup_stm32f40_41xxx.o
    0x200011e0   0x00000400   Zero   RW            1    STACK               startup_stm32f40_41xxx.o


==============================================================================

Image component sizes


      Code (inc. data)   RO Data    RW Data    ZI Data      Debug   Object Name

        84         22          0         14       1520       1774   main.o
       228         22          0          0          0       1777   misc.o
        64         26        392          0       1536        772   startup_stm32f40_41xxx.o
       324         42         37         24          0       2654   stm32f4_discovery.o
      3124        220          0         76        120      10219   stm32f4_discovery_audio_codec.o
       528          6          0          0          0       4813   stm32f4xx_dac.o
       932         32          0          0          0       6201   stm32f4xx_dma.o
       284         10          0          0          0       2207   stm32f4xx_exti.o
       604         36          0          0          0       3873   stm32f4xx_gpio.o
      1064         26          0          0          0       7935   stm32f4xx_i2c.o
        84          8          0          0          0       1503   stm32f4xx_it.o
      1416         48          0         16          0      10803   stm32f4xx_rcc.o
      1012         22          0          0          0       6569   stm32f4xx_spi.o
       140         12          0          0          0       1499   stm32f4xx_syscfg.o
       564         50          0         20          0     273167   system_stm32f4xx.o
       256          4          0          0          0       1505   usb_bsp.o
      4222         16          0          0          0      12440   usb_core.o
       894          0          0          0          0       4192   usb_dcd.o
      2000         20          0          0          0       4823   usb_dcd_int.o
       644         52          0        181       1600      24915   usbd_audio_core.o
       328         10          0         36          0       4580   usbd_audio_out_if.o
       702          0          0         48          0       4932   usbd_core.o
       344        168          0         60          0       3368   usbd_desc.o
       244          0          0          0          0       2486   usbd_ioreq.o
      1744         50          0         13        200       5157   usbd_req.o
       132         14          0         28          0      28096   usbd_usr.o

    ----------------------------------------------------------------------
     21964        916        464        524       4976     432260   Object Totals
         0          0         32          0          0          0   (incl. Generated)
         2          0          3          8          0          0   (incl. Padding)

    ----------------------------------------------------------------------

      Code (inc. data)   RO Data    RW Data    ZI Data      Debug   Library Member Name

        90          0          0          0          0          0   __dczerorl2.o
         8          0          0          0          0         68   __main.o
        52          8          0          0          0          0   __scatter.o
        28          0          0          0          0          0   __scatter_zi.o
        12          0          0          0          0         72   exit.o
         6          0          0          0          0        152   heapauxi.o
         0          0          0          0          0          0   indicate_semi.o
         2          0          0          0          0          0   libinit.o
         2          0          0          0          0          0   libinit2.o
         2          0          0          0          0          0   libshutdown.o
         2          0          0          0          0          0   libshutdown2.o
         8          4          0          0         96         68   libspace.o
         0          0          0          0          0          0   rtentry.o
        12          0          0          0          0          0   rtentry2.o
         6          0          0          0          0          0   rtentry4.o
         2          0          0          0          0          0   rtexit.o
        10          0          0          0          0          0   rtexit2.o
        12          4          0          0          0         68   sys_exit.o
        74          0          0          0          0         80   sys_stackheap_outer.o
         2          0          0          0          0         68   use_no_semi.o

    ----------------------------------------------------------------------
       336         16          0          0        100        576   Library Totals
         6          0          0          0          4          0   (incl. Padding)

    ----------------------------------------------------------------------

      Code (inc. data)   RO Data    RW Data    ZI Data      Debug   Library Name

       330         16          0          0         96        576   c_w.l

    ----------------------------------------------------------------------
       336         16          0          0        100        576   Library Totals

    ----------------------------------------------------------------------

==============================================================================


      Code (inc. data)   RO Data    RW Data    ZI Data      Debug   

     22300        932        464        524       5076     429976   Grand Totals
     22300        932        464        320       5076     429976   ELF Image Totals (compressed)
     22300        932        464        320          0          0   ROM Totals

==============================================================================

    Total RO  Size (Code + RO Data)                22764 (  22.23kB)
    Total RW  Size (RW Data + ZI Data)              5600 (   5.47kB)
    Total ROM Size (Code + RO Data + RW Data)      23084 (  22.54kB)

==============================================================================

